:07FD5F009022AA7408F022B3
:0DD7F8009022A7EDF0A3EBF09022A6EFF039
:10D80500BFFF09E4F0786CE6A3F0800B9022A6E058
:10D81500C3950B4002D3229022A7E0FFC3950D408C
:10D8250002D3229022A8E0FEF46025EE5490600217
:10D83500D3229022A8E0FE541FC3950B4002D322A9
:10D84500EE54E0700B9022A9E0C3950D4002D3225F
:10D855003018359022A8E0FE54F07016745C2EF84E
:10D86500A3E0FE66600CEE04FE9022A8E0242CF8EE
:10D87500A6069022A6E0FE246CF8E66F600AA3E0F7
:10D8850004FF744C2EF8A6079022A8E0FF54E09000
:10D8950022AAF070219022A9E0FEEF541FFF245C1C
:10D8A500F8A606E50B24031313543FFEEF13135498
:10D8B5003F2EF511807E9022AAE0FF6420703E3055
:10D8C50012179022A9E0C3945B4003745AF0E50B4C
:10D8D50014FE9022A8E05E80129022A9E0C3942055
:10D8E5004003741FF09022A8E0541FFE243CF874F6
:10D8F5008056F6743C2EF8A3E046F68037EF644078
:10D9050070169022A8E0301204547F8002541F2420
:10D915003CF8747F56F6801C9022AAE0646070146F
:10D925009022A8E0301204547F8002541F243CF852
:10D93500748046F69022A6E0246CF8A3E0FF6660AA
:10D945000E9022A6E0FEA607EE1313543FF511D262
:10D95500C4D2C1D2C012FD5F9022A8E0FF30E70417
:10D96500D2C18002C2C19022A812D9CF70EA12FD9D
:10D975005F9022A9E0FF30E704D2C18002C2C190C6
:10D9850022A912D9CF70EA12FD5F9022A6E0FF30DE
:10D99500E704D2C18002C2C19022A612D9EB70EA77
:10D9A50012FD5F9022A7E0FF30E704D2C18002C2DA
:10D9B500C19022A712D9EB70EAC2C412FBBE12FBBA
:09D9C500BED2C4301802D219C30D
:10D9CE0022EF25E0F0C2C012FBBE12FBBED2C01287
:10D9DE00FBD612FBD69022AAE014F0E022EF25E04F
:10D9EE00F0C2C012FBBE12FBBED2C012FBD612FB9F
:09D9FE00D69022AAE014F0E02208
:10E67200E49022A5F09022A5E0C3950B400302E7A7
:10E6820005300C5FE0FF246CF8E6FDE0FE541FFB52
:10E69200745C2EF8E69022A9F012D7F89022A5E039
:10E6A200FF243CF8E630E707EF541F4460800890EF
:10E6B20022A5E0541F4440FBE49022A9F0FD7FFF15
:10E6C20012D7F8301402D20D9022A5E0FF541F4455
:10E6D20020FB743C2FF8E6547F9022A9F0E4FD7FE2
:10E6E200FF80119022A5E0FF246CF8E6FDE4902261
:10E6F200A9F07BFF12D7F812F6D99022A5E004F018
:03E7020002E677B5
:01E7050022F1
:10E5DA00434F5059524947485420313939392D321D
:10E5EA00303036204E4554574F524B2054454348FD
:10E5FA004E4F4C4F4749455320494E4320414C4CBE
:10E60A00205249474854532052455345525645448F
:10E61A00200024534D206D586E20566964656F2F73
:10E62A00417564696F20240024446174653A20327C
:10E63A003030372F30352F30332031373A30393AAE
:10E64A003034202400245265766973696F6E3A204B
:10E65A00312E3220240024494E3A20002024244F0F
:08E66A0055543A200020240061
:0CF7DC004322B13136004322AE3136002A
:10FBBE000000000000000000000000000000000037
:08FBCE0000000000000000220D
:10FBD600C0E0740E000000000000000000000000FD
:06FBE600D5E0F1D0E022A1
:0EFC8F00C0E0742500000000D5E0F9D0E022AE
:10F6D900C0E0C0F075F00A74FD00000000000000F1
:10F6E9000000000000000000000000000000000011
:0CF6F90000D5E0E5D5F0E0D0F0D0E02234
:10F80300C0E074FD000000000000000000000000E4
:10F813000000000000000000000000000000D5E030
:06F82300E3DFDFD0E0226C
:10FC600061646D696E003336303000506F7274001D
:10DB93009022A712CC769022AAE029F9E43AFA025D
:10DBA300C90290229C12CC7690229FE0F582758365
:10DBB3000002C91B781AEEF608EFF6EE229022A5B2
:10DBC300E075F010A4AEF0229022A7E025E025E056
:10DBD3002468F582E43421F58322E0FAA3E0FBFF15
:10DBE3007C007D08AE0202C98E9022A712CC7690EB
:10DBF30022AA2290229BE024C4F582E43421F583F7
:10DC03002290229DE024B3F582E43421F58322E0BF
:10DC130004F0E0C394042290229BE0242CF582E4D8
:10DC23003421F583229022A6E0FF14F0EF22902204
:10DC3300A6E0FF14F0EF2218F6E49022A7F022905A
:10DC430022A7E0C3950B22EEF0A3EFF0A302CC963C
:10DC5300E0FEA3E0FF7C007D0C12C97CEF2430FFC3
:10DC6300EE343AFE227BFF9022A802CC969022A6A5
:10DC73007420F0229022A7E004F022EFF0A3742096
:10DC8300F022781BE6FF9022A7E022EFF07C007DD4
:10DC930008AF03AE0212C98EAF05EF2218F6A374C4
:10DCA30020F0227E00781BE6FFE4FCFD22E004F076
:10DCB300E0C3941022E024ABF582E43421F58322FF
:10DCC300E024AFF582E43421F58322E02451F58288
:10DCD300E43421F58322E024C0F582E43421F58382
:10DCE300229022A7E075F004A42275F00A84E5F0DF
:10DCF30024302274C0F0A374A8F0A37401F0A3220B
:0FDD0300F582E43421F5832275F00A842430225E
:06EE66009022A812DC4A14
:10EE6C00E4FFFE9022ADE0FDC3EF9D7480F86E9838
:10EE7C00501B9022AA12CC768F828E8312C91BFD56
:10EE8C00747C2FF8A6050FBF00010E80D69022A827
:10EE9C00E0FEA3E0FF7D7C9022ADE0FB12DE57E4A8
:02EEAC0033FF32
:01EEAE002241
:0EE3C8009022A8EEF0A3EFF0A3EDF0A3EBF08F
:10E3D600E4A3F0A3F09022ABE0FFC39022ADE09F50
:10E3E6007480F89022ACE0648098400302E47FE5F4
:10E3F6000B1313543FFF9022AAE0FEEF8EF0A4FB0E
:10E40600AAF09022ACE0FEA3E0FF7C007D0412C9D6
:10E416008EEB2FFFEA3EFEEF7802C333CE33CED823
:10E42600F92468F58274213EF58312CC21C004C01C
:10E4360005C006C0079022ABE0FFA3E0FCA3E0FD09
:10E44600C3EF9DFFE49CCF24FFCF34FFFE7C007D0D
:10E456000412C98EED75F008A4F9D007D006D005D0
:10E46600D004F812CBFBE0247CF8A6079022ACE49B
:10E4760075F00112C9C402E3DB9022A8E0FEA3E016
:0EE48600FF7D7C9022ABE0FB12DE57E433FFFB
:01E494002265
:05DFE7009022A5EFF0FF
:10DFEC0012DBC42420781BF6E43E12DC9F12DC28E2
:10DFFC00600E7A00796C12E0E7700512F6D980EDAC
:10E00C0012DBC02460781BF6EE340612DC9F12DCA7
:10E01C0028600E7A00795C12E0E7700512F6D98060
:10E02C00ED12DBC024A0781BF6EE340C12DC9F1230
:10E03C00DC28600E7A00793C12E0FB700512F6D9F0
:10E04C0080ED12DBC024E0781BF6EE341212DC9F5C
:10E05C0012DC28601E781AE6FE08E6FF7B017A21A6
:10E06C00793D9022ADE50BF012EE66EF700512F6DD
:10E07C00D980DD12DBC02420781BF6EE341912DCBB
:10E08C009F12DC28600E7A00798E12E0FB7005126C
:10E09C00F6D980ED12DBC02460781BF6EE341F1825
:10E0AC00F6E49022A7F09022A67420F012DC2860EF
:10E0BC0021A3E0FD850BF0A4FF781AE6FA08E62F01
:10E0CC00FFE5F03AFEAB0B12E3C8EF700512F6D980
:0AE0DC0080DA9022A712DC1240CC7B
:10E0E60022781AE6FE08E6FF7B009022ADE50BF0EB
:10E0F60012EE66EF22781AE6FE08E6FF7B00902213
:09E10600ADE50BF012EE66EF220C
:05D0B6009022A5EFF03F
:10D0BB0012DBC42420781DF6E43E12DC3A12DC426B
:10D0CB00503912DC7012DC31602C12D31270F63036
:10D0DB00181C9022A7E0FF246CF8E6FD781BE66D88
:10D0EB007001E46009E604FE744C2FF8A60612DC0E
:10D0FB0085246CF8A60712DC7780C29022A512DB80
:10D10B00C32460781DF6EE340612DC3A12DC425072
:10D11B003912DC7012DC31602C12D31270F630181D
:10D12B001C9022A7E0FF245CF8E6FD781BE66D70EF
:10D13B0001E46009E604FE742C2FF8A60612DC85C8
:10D14B00245CF8A60712DC7780C29022A512DBC301
:10D15B0024A0781DF6EE340C12DC3A12DC42501D82
:10D16B0012DC7012DC31601012D34212DBB770F399
:10D17B0012DC87243CF8A60712DC7780DE9022A510
:10D18B0012DBC324E0781DF6EE341212DC3A12DC0B
:10D19B0042502312DC7012DC31601612D34212DBC8
:10D1AB00B770F312DC87243DF582E43421F583EF6D
:10D1BB00F012DC7780D89022A512DBC32420781DD7
:10D1CB00F6EE341912DC3A12DC42503612DC7012D5
:10D1DB00DC316029A3E0781D26FFE41836FE12DE51
:10D1EB002212DBB770E912DC87FE248EF8A60774D7
:10D1FB008E2EF8E6FF74572E12DD03EFF012DC775C
:10D20B0080C59022A512DBC32460781DF6EE341F77
:10D21B0012DC3A12DC42400302D31112DC7012DC36
:10D22B0031700302D30BA3E075F004A4FF781CE666
:10D23B00FC08E62FFFE5F03CFE12DE2212DBB77096
:10D24B0014FEE6FFE4FCFDFBFAF9780112CA991211
:10D25B00DBCB12CC3912DCE4240112D328702F1251
:10D26B00DBCBC083C08212CC2DC000C001C002C07A
:10D27B000312DCA6FBFA7901F812CA99D003D0028B
:10D28B00D001D00012CA8CD082D08312CC3912DCE0
:10D29B00E4240212D328702F12DBCBC083C082127E
:10D2AB00CC2DC000C001C002C00312DCA6FB7A016A
:10D2BB00F9F812CA99D003D002D001D00012CA8C4F
:10D2CB00D082D08312CC3912DCE42403FFE435F096
:10D2DB00FEEF781D26FFEE1836FE12DE2212DBB7AC
:10D2EB00600302D22912DBCBC083C08212CC2DC0CB
:10D2FB000012DCA6D00012CA8CD082D08312CC399B
:06D30B0012DC7702D21EC5
:10D3110022A3E0781D26FFE41836FE12DE22781AD9
:10D32100EEF608EFF6EE22FFE435F0FEEF781D266B
:10D33100FFEE1836FE12DE22781AEEF608EFF6EE50
:0FD3410022A3E0781D26FFE41836FE12DE22221A
:03F84E009022A560
:10F8510012DC7E9022A6E0FF14F0EF60139022A547
:10F86100E0FD7F027E0012DDF8400512F6D980E34B
:01F871002274
:10F872009022A67420F09022A6E0FF14F0EF60110F
:10F882007F027E0012DE22781912DBB970E8E6FFF1
:03F89200227FFFD3
:01F895002250
:03F896009022A518
:10F8990012DC7E9022A6E0FF14F0EF60139022A5FF
:10F8A900E0FD7F037E0012DDF8400512F6D980E302
:01F8B900222C
:10F8BA0090229A7420F090229AE0FF14F0EF6011DF
:10F8CA007F037E0012DE22781A12DBB970E8E6FFA7
:03F8DA00227FFF8B
:01F8DD002208
:10F2310090229A7420F090229AE0FF14F0EF60106F
:10F241007DFE7F017E3A12DDF8400512F6D980E697
:10F2510090229A7420F090229AE0FF14F0EF60104F
:10F261007DCA7F027E3A12DDF8400512F6D980E6AA
:01F27100227A
:10F2720090229A7420F090229AE0FF14F0EF60102E
:10F28200E4FD7F017E3A12DDF8400512F6D980E6F0
:10F2920090229A7420F090229AE0FF14F0EF60100E
:10F2A200E4FD7F027E3A12DDF8400512F6D980E6CF
:01F2B2002239
:10EC2100C21AC21B90229A7420F090229AE0FF141B
:10EC3100F0EF601A7F017E3A12DE22781A12DBB9F8
:10EC410070E818F608E664FE184670DED21A9022C3
:10EC51009A7420F090229AE0FF14F0EF601A7F027C
:10EC61007E3A12DE22781A12DBB970E818F608E64D
:0CEC710064CA184670DED21BA21B821A77
:01EC7D002274
:10F3EB00E49022A6F09022A57420F09022A5E0FFD5
:10F3FB0014F0EF601CA3E0FD2403FFE4343AFE7429
:10F40B00AB2D12DCBBE0FD12DDF8400512F6D98006
:09F41B00DA9022A612DC1240CCAA
:01F4240022C5
:10EEF700E490229BF090229A7420F090229AE0FFEF
:10EF070014F0EF601DA3E02403FFE4343AFE12DEA1
:10EF170022781A12DBB970E3E6FF90229B12DCB865
:10EF2700EFF090229AE07006A312DCB8E4F090228A
:06EF37009B12DC1240BF3A
:01EF3D0022B1
:10F42500E49022A6F09022A57420F09022A5E0FF9A
:10F4350014F0EF601CA3E0FD2400FFE43438FE74F3
:10F44500AF2D12DCC6E0FD12DDF8400512F6D980BD
:09F45500DA9022A612DC1240CC70
:01F45E00228B
:10EF3E00E490229BF090229A7420F090229AE0FFA7
:10EF4E0014F0EF601DA3E02400FFE43438FE12DE5F
:10EF5E0022781A12DBB970E3E6FF90229B12DCC313
:10EF6E00EFF090229AE07006A312DCC3E4F0902238
:06EF7E009B12DC1240BFF3
:01EF8400226A
:10F45F00E49022A6F09022A57420F09022A5E0FF60
:10F46F0014F0EF601CA3E0FD2407FFE4343AFE74B0
:10F47F00512D12DCD1E0FD12DDF8400512F6D980D6
:09F48F00DA9022A612DC1240CC36
:01F498002251
:10EF8500E490229BF090229A7420F090229AE0FF60
:10EF950014F0EF601DA3E02407FFE4343AFE12DE0F
:10EFA50022781A12DBB970E3E6FF90229B12DCCEC1
:10EFB500EFF090229AE07006A312DCCEE4F09022E6
:06EFC5009B12DC1240BFAC
:01EFCB002223
:10F49900E49022A6F09022A57420F09022A5E0FF26
:10F4A90014F0EF601CA3E0FD240BFFE4343AFE7472
:10F4B900C02D12DCDCE0FD12DDF8400512F6D98022
:09F4C900DA9022A612DC1240CCFC
:01F4D2002217
:10EFCC00E490229BF090229A7420F090229AE0FF19
:10EFDC0014F0EF601DA3E0240BFFE4343AFE12DEC4
:10EFEC0022781A12DBB970E3E6FF90229B12DCD96F
:10EFFC00EFF090229AE07006A312DCD9E4F0902294
:06F00C009B12DC1240BF64
:01F0120022DB
:10F0E300E49022A6F09022A57420F09022A5E0FFE0
:10F0F30014F0EF601CA3E0FD2410FFE4343AFE7427
:10F10300C42D12DBFCE0FD12DDF8400512F6D980B8
:10F11300DA9022A612DBF9E060089022A612DCB096
:02F1230040C3E7
:01F1250022C7
:10ED2C00E490229BF090229A7420F090229AE0FFBB
:10ED3C0014F0EF601AA3E02410FFE4343AFE12DE64
:10ED4C0022781A12DBB970E3E6FF12DBF6EFF090D3
:10ED5C00229AE06007A312DBF9E0700712DBF6E4FD
:10ED6C00F0800890229B12DCB040BA12DBF6E4F083
:01ED7C002274
:10F12600E49022A6F09022A57420F09022A5E0FF9C
:10F1360014F0EF601CA3E0FD2420FFE4343AFE74D3
:10F146002C2D12DC20E0FD12DDF8400512F6D980E8
:10F15600DA9022A612DC1DE060089022A612DCB02E
:02F1660040C3A4
:01F168002284
:10EE1B00E490229BF090229A7420F090229AE0FFCB
:10EE2B0014F0EF601AA3E02420FFE4343AFE12DE64
:10EE3B0022781A12DBB970E3E6FF12DC1AEFF090BE
:10EE4B00229AE06007A312DC1DE0700612DC1AE4C4
:0AEE5B00F02290229B12DCB040BBB5
:01EE6500228A
:08EC7E009022A5EEF0A3EFF0D7
:10EC8600E49022A8F09022A77420F09022A7E0FF3B
:10EC960014F0EF60249022A512DC539022A8E0FD28
:10ECA6007A002FFFEA3EFE74B32D12DC0AE0FD1255
:10ECB600DDF8400512F6D980D29022A812DC07E0D2
:0EECC600600C9022A8E004F0E0C3940C40B76C
:01ECD400221D
:08EB600090229AEEF0A3EFF001
:10EB6800E490229DF090229C7420F090229CE0FF7B
:10EB780014F0EF602090229A12DC5390229DE02F2F
:10EB8800FFEC3EFE12DE22781612DBB970DDE6FFDE
:10EB980012DC04EFF090229CE06007A312DC07E08F
:10EBA800700712DC04E4F0800C90229DE004F0E091
:0AEBB800C3940C40B012DC04E4F03A
:01EBC2002230
:03F8DE0090229ADB
:10F8E10012DC7E90229BE0FF14F0EF601390229ACD
:10F8F100E0FD7FF07E3F12DDF8400512F6D980E38E
:01F9010022E3
:10F9D90090229A7420F090229AE0FF14F0EF6011BF
:10F9E9007FF07E3F12DE22781A12DBB970E8E6F565
:01F9F9000B02
:01F9FA0022EA
:03F9020090229AB6
:10F9050012DC7E90229BE0FF14F0EF601390229AA8
:10F91500E0FD7FF17E3F12DDF8400512F6D980E368
:01F9250022BF
:10F9FB0090229A7420F090229AE0FF14F0EF60119D
:10FA0B007FF17E3F12DE22781A12DBB970E8E6F541
:01FA1B000DDD
:01FA1C0022C7
:03F9260090229A92
:10F9290012DC7E90229BE0FF14F0EF601390229A84
:10F93900E0FD7FF27E3F12DDF8400512F6D980E343
:01F94900229B
:10F94A0090229A7420F090229AE0FF14F0EF60134C
:10F95A007FF27E3F12DE22781A12DBB970E8E624C3
:03F96A00FF920CFD
:01F96D002277
:03F96E0090229A4A
:10F9710012DC7E90229BE0FF14F0EF601390229A3C
:10F98100E0FD7FF37E3F12DDF8400512F6D980E3FA
:01F991002253
:10F9920090229A7420F090229AE0FF14F0EF601304
:10F9A2007FF37E3F12DE22781A12DBB970E8E6247A
:03F9B200FF9212AF
:01F9B500222F
:07FD4700C2C712FCE4D2C7A1
:01FD4E002292
:10E89800E490229AF0FB90229AE0FF746C2BF8A681
:10E8A80007745C2BF8A607743C2BF8301204760A20
:10E8B80080027605743D2BF582E43421F58374508B
:10E8C800F0748E2BF8E4F6748E2BF8E6FF74572B51
:10E8D80012DD03EFF0EB12DBCF12CC45FFFFFFFF99
:10E8E80090229AE004F0E0C3950D4002E4F00BEBAF
:10E8F800641070A2E490229AF090229AE0FFC394E8
:0EE9080064500B12DFE790229AE004F080EBDF
:01E9160022DE
:10D5BA0012F9D912F9FB12F94A12F99212FD477EB1
:10D5CA00007816EEF608EFF664236071E418F608A0
:10D5DA00F6FF12DE22781812DBB97008E6781646D2
:10D5EA00F608E6F67F017E0012DE22781812DBB911
:10D5FA00700AE6FF7816E6F608E64FF67816B65A87
:10D60A001008B6CE0C12F8BA8F08E4FF12D0B68012
:10D61A002C750801AF0812F896750B10750D10C21B
:10D62A000CC212AF0B12F8DEAF0D12F902A20CE413
:10D63A0033FF12F926A212E433FF12F96E7817E6C5
:10D64A0064CE700418E6645A605212E89812F272B4
:10D65A00750801AF0812F8967F0312F84E902299C6
:10D66A007420F0902299E0FF14F0EF600F7D5AE4E5
:10D67A00FFFE12DDF8400512F6D980E79022997470
:10D68A0020F0902299E0FF14F0EF60107DCE7F0128
:10D69A007E0012DDF8400512F6D980E6E490229960
:10D6AA00F0902299E0FFC39410501174572F12DDA5
:10D6BA00037401F0902299E004F080E5E50B12DD95
:10D6CA000BF50EE50B12DCEDF50FE4F510FB7A0015
:10D6DA00790E12DC6A0B7A2279AE12FA83E50D1200
:10D6EA00DD0BF513E50D12DCEDF514E4F515FB7A07
:10D6FA0000791312DC6A0B7A2279B112FA83C21406
:10D70A00C20AC203C201C20FC20BC204C210C211B2
:10D71A00C202C20DE4902156F0902150F090214EA1
:10D72A00F09021A9F09021AAF09021A8F090216709
:10D73A00F012EC21500302D7E59021AB12DCF6740B
:10D74A001EF012F3EB90215174FFF0A3F0A3F0E462
:10D75A00A3F012F45F9021C012DCF6F012F499E4FF
:10D76A009021AFF0A3F0A3F0A3F012F4257AFC798C
:10D77A006012DC687B017A2179C412FA8312F0E321
:10D78A007AFC796612DC687B017A21792C12FA8399
:10D79A0012F126E49021B3F0902299F07BFF7AFCF3
:10D7AA00796B12DC6A7B017A2179B312FA839022AF
:10D7BA0099E0FC04FE12DD0B9021B7F0EE12DCEDCD
:10D7CA00A3F0E4A3F0ECFF7E0012EC7E902299E035
:10D7DA0004F0E0C3942040C402F23112EEF712EFD3
:0DD7EA008512EFCC12ED2C12EE1B12EF3E5B
:01D7F700220F
:06EA83009022A512DC4AFE
:10EA89009022A512DBDD9022AAEFF0AF0312DBE39F
:10EA9900AF05EF12CCBFEABB00EAC301EACB02EA39
:10EAA900D203EAD904EAE005EAE706EAEE0700003C
:10EAB900EAF612DB93440102EAF312DB9344020201
:10EAC900EAF312DB934404802112DB934408801A91
:10EAD90012DB934410801312DB934420800C12DB69
:0DEAE900934440800512DB93448012C9481D
:01EAF60022FD
:06E792009022A512DC4AF2
:10E798009022A512DBDD9022AA12DC8E12CCBFE7F4
:10E7A800C300E7CE01E7D902E7E303E7ED04E7F7A3
:10E7B80005E80106E80B070000E81612DBEC12DB9F
:10E7C8009C54FE02E81312DBEC12DB9C54FD02E8B9
:10E7D8001312DBEC12DB9C54FB803012DBEC12DBF7
:10E7E8009C54F7802612DBEC12DB9C54EF801C1241
:10E7F800DBEC12DB9C54DF801212DBEC12DB9C5446
:0EE80800BF800812DBEC12DB9C547F12C94863
:01E8160022DF
:06E4950090229A12DC4AFD
:10E49B0090229A12DBDD90229F12DC8E12CCBFE40D
:10E4AB00C600E4D501E4E402E4F303E50204E5115C
:10E4BB0005E52006E52F070000E53D12DBA554011D
:10E4CB009022A0F07002C322D32212DBA55402903B
:10E4DB0022A0F07002C322D32212DBA55404902297
:10E4EB00A0F07002C322D32212DBA554089022A005
:10E4FB00F07002C322D32212DBA554109022A0F09D
:10E50B007002C322D32212DBA554209022A0F070FC
:10E51B0002C322D32212DBA554409022A0F070023A
:10E52B00C322D32212DBA554809022A0F07002C329
:02E53B0022D3E9
:01E53D0022BB
:10DD1200D2B6D2B730B61D30B71A00000000C2B674
:10DD220000000000000000000000000000000000F1
:10DD3200C2B7D322C322C2B6000000000000000016
:10DD42000000000000000000D2B700000000000048
:10DD520000000000000000000000D2B622C2B6801F
:10DD620002D2B600000000000000000000D2B7009E
:10DD7200000000000000000000000000000000C2DF
:10DD8200B722C0027A083392B600000000D2B70070
:10DD9200000000000000000000000000000000C2BF
:10DDA200B700DAE2D2B60000000000000000000076
:0DDDB200D2B70000000000000000000000DB
:10DDBF000000000000A2B6C2B7B3D00222C0027AA0
:10DDCF0008D2B600000000000000000000000000B4
:10DDDF00000000D2B700000000000000000000A209
:10DDEF00B633C2B7DADDD0022212DD12502474A08E
:10DDFF0012DD84501AEE12DD845014EF12DD8450C0
:10DE0F000EED12DD84500812DD3812F6D9D322122E
:10DE1F00DD382212DD12502A74A012DD845020EE5C
:10DE2F0012DD84501AEF12DD84501412DD125012DD
:10DE3F0074A112DD84500812DDCC12DD63FFD31202
:10DE4F00DD387E0040011E22EDF912DD12502774DD
:10DE5F00A012DD84501DEE12DD845017EF12DD8409
:10DE6F005011E712DD84500B09DBF712DD3812F683
:07DE7F00D9D32212DD382285
:10802600E475F00112CA1290000712C9DAFFAEF029
:10803600229022A312CC769000032290229B12CC8F
:05804600769000052208
:10ED7D009022A6EDF09022A312CC9612F67EEF60B3
:10ED8D00057EFF7FFF229022A6E0FF12803712C979
:10ED9D00DAFDACF012CC9F8D828C83EF12C95A1222
:10EDAD00803712802690000312C9DAC39FE5F09ECA
:0FEDBD004009128037E4F5F012CA5FE4FEFF222E
:06EDCC0090229B12CC9680
:10EDD20012FB72EF60057EFF7FFF221280411280DC
:10EDE2003012CC9F8F828E8312C91BFF90229EE429
:10EDF200F0A3EFF012804112802690000512C9DACA
:10EE0200C39FE5F09E4009128041E4F5F012CA5F0B
:08EE120090229EE0FEA3E0FF48
:01EE1A0022D5
:10FB720090000512803090000312C9DAB50708E53B
:0AFB8200F0B506037F01227F002288
:10F67E009000031280300FBF00010E90000712C9D8
:10F68E00DAB50707EEB5F003E4FEFF90000512C9E8
:0DF69E00DAB50707EEB5F0037F01227F000B
:01F6AB00223C
:08FD4F00C289D2A843910422ED
:0CFC9D0012FC8FC295902801E0FFD29568
:01FCA9002238
:0380030002FD7308
:03FD7300D2133276
:10F57D00301333C21312FC9DAE07EEF4C4135407BF
:10F58D00FC902810E020E20474082CFCEE541FFEC1
:10F59D00AF04FDEC541FFB9022A9EEF012D7F8300A
:06F5AD001404D203D20198
:01F5B3002235
:0CF7E80049200001200900000000010081
:10F3AF00E4FCFDFE12CC0EA804A905AA06AB07903B
:10F3BF00210902CC21E4FC12CA8C90210902CC391C
:10F3CF0012CC2DC302CBEA12CC2D12CBB6E4FBFA32
:0CF3DF00F9F8C302CBEA90229D02CC2179
:09FCE400C296902801E0FFD296BF
:01FCED0022F4
:10F64F0090211974FFF090211112CC45003F3F3FDC
:10F65F0090210D12CC45003F3F3F90210912CC4520
:0FF66F00003F3F3F90211512CC45003F3F3F2207
:10E53E0012F3BE90211512CC2D12CBD0902299122F
:10E54E00CC3990229D12CC4500000001E49022A10E
:10E55E00F0E4FFFEFDFC90229912F3CF606590224D
:10E56E00A274FFF012F3E590229912F3D6602612F0
:10E57E00F3E590210912F3D69022A17005E0A3F0E5
:10E58E008005E04480A3F07B017A2079009022A2DE
:10E59E00E0FD12ED7D12F3E512CBDD90229912CC47
:10E5AE002D12CBB690229912CC3912F3E5780112C6
:10E5BE00CC0EE4FC90229D12CC399022A1E004F006
:0CE5CE0002E55F12F3BE90211502CC396B
:10EA0D00C2C712FCE4AB07E4FAF9F812F3BEE4FF57
:10EA1D0012F3C4D2C7C2C612FCE4780812F3AFE4F5
:10EA2D00FE12F3C4D2C6C2C512FCE4781012F3AFC5
:10EA3D00E4FD12F3C5D2C512F3BE90211512F3CF2A
:10EA4D00601F90210D12CC2190210912F3CF70116E
:10EA5D0090211112CC2190210D12F3CF700312E5EC
:10EA6D003E90210D12CC2190211112CC3912F3BE02
:06EA7D0090210D02CC39CE
:10FC2B007D0A7F0312F78750087F0312FD6612EAE5
:02FC3B000D2298
:0DFCAA00902805EFF0D2B5C2B574FFF0222E
:0AFCEE00D2B412FCAA7F0202F80350
:06FD6D00C2B412FCAA2240
:09FD3E007F0112FD6D0F02F803B4
:10FB3B00EFD394025015EFB40205ED24C08003ED12
:0CFB4B002480FF12FD6D7F0212F80322DF
:10F3710090229AEFF0C36480948A401EE0FF75F0FA
:10F381000A12C8E02430FF12FCEE90229AE0FF75C9
:10F39100F00A12C8E0AFF0EF80097F2012FCEE9076
:0EF3A100229AE02430FF12FCEE7F2002FCEEE8
:10EAF70090229AEFF0C39464401CE075F06484247C
:10EB070030FF12EB5875F06484E5F012EB4975F0AD
:10EB17000A84E5F0802590229AE0C3940A7F20407A
:10EB27000E12EB5812EB4975F00A84E5F0800C12CF
:10EB3700FCEE7F2012FCEE90229AE02430FF12FCBC
:10EB4700EE2275F00A842430FF12FCEE90229AE040
:09EB57002212FCEE90229AE02249
:06FAA50090229A12CC969B
:10FAAB0090229AE475F00112CC7F12C90290229D2C
:0AFABB00F06007E0FF12FCEE80E6A9
:01FAC500221E
:10F09F007F1412F8037F3812FD6D7F0512F0D57FB4
:10F0AF003812FD6D7F0212F0D57F0612FD6D7F02C3
:10F0BF0012F8037F0E12FD6D7F0212F8037F01120B
:10F0CF00FD6D0F02F80312F8037F3812FD6D7F02FA
:04F0DF0012F80322FE
:10CD84004E6574776F726B205465636820496E63D7
:10CD94002E002D2D2D534D007800205626412D2D8B
:10CDA4000020562D2D2D2D004F55543A2000764944
:10CDB4004E3A200061494E3A200042414420494EF7
:10CDC4002056414C55452000424144204F555420A3
:10CDD40056414C5545002020494E3A2000566F6C70
:10CDE4003A20002020302000644220006D757465D4
:10CDF40000202020200042414420556E69742041C7
:10CE040064640031292A39363030203229203438FC
:10CE1400303020003329203234303020342920317E
:10CE24003230302000312920393630302032292A5E
:10CE3400343830302000312920393630302032293E
:10CE44002034383030200033292A32343030203432
:10CE54002920313230302000332920323430302040
:10CE640034292A3132303020003129204E62206F9B
:10CE74006620496E70757473003229204E62206FEB
:10CE840066204F7574707574730033292056696475
:10CE9400656F202620417564696F00342920484459
:10CEA4005456202020202020202020004E62206F75
:10CEB4006620496E707574733A20004E62206F6666
:10CEC400204F7574707574733A0031293E56696445
:10CED400656F202620417564696F003229205669E8
:10CEE40064656F204F6E6C79202020003129205614
:10CEF4006964656F202620417564696F0032293E9C
:10CF0400566964656F204F6E6C79202020003129AA
:10CF14003E4844545620456E61626C656400322973
:10CF240020484454562044697361626C656400313E
:10CF340029204844545620456E61626C6564003271
:10CF4400293E484454562044697361626C65640008
:10CF5400424144204E622E20496E70757473005015
:10CF64006C6561736520776169742E2E2E20200014
:10CF7400424144204E622E204F75747075747300C4
:10CF8400332920536574205363616E204D6F6465AB
:10CF940000332920323430302034293E31323030CD
:10CFA400200033293E3234303020342920313230CD
:10CFB400302000312920393630302032293E3438AF
:10CFC4003030200031293E393630302032292034A7
:10CFD40038303020002800293A0053656C656374AA
:10CFE40020506F7274005F0043757272656E742016
:10CFF40074696D653A004E65772074696D653A20F1
:10D004002020200053657175656E6365205363614C
:10D014006E00697320616374697665004D656D6F98
:10D02400727920536176653A20004D656D6F72798F
:10D0340020526563616C6C3A0053657420616C6CBA
:10D0440020494E3A200031292053657420426175ED
:10D054006420526174650032292053657420556E32
:10D0640069742041646472001B8237383984818377
:10D07400343536852A303132330D566964656F2074
:10D084002620417564696F00566964656F206F6E70
:10D094006C7920202000417564696F206F6E6C7973
:10D0A40020202000566F6C756D652C204D757465BD
:02D0B40020005A
:10E209007824E67825F67824E4F6788C762708765B
:10E2190010227816E6FF12FBEC7817EFF622782524
:10E22900E6FF7824E675F00AA4221511E50B24030C
:10E239001313543F222EF582E435F0F583E5822449
:10E249003CF582E5833421F583EFF0227825E6FF5A
:10E259007824E6FE75F00AA42F243BF8E62275F02F
:10E2690002A4FFC3E5119FE5F06480F87480982249
:10E2790078252614FF7826E675F00AA47827262241
:10E28900FFC3E5119F25E025E0227817E6FF24D09A
:10E2990022FFC3E5119FFFEF25E025E022750C1150
:10E2A9007817E624D07924F722E50B141313543F89
:10E2B90022E51125E025E022788C760F0876A02248
:10E2C9007817E6D3940A227817E6D3940522902288
:10E2D900987409F0750C0B2278252614541F229086
:10E2E9002284E004F0229022987424F0750C2322F1
:0BFCC3001FEFC3950B40028001D3220D
:0AFCF800EFD3940F40028001D322E5
:0BFCCE001FEFC3950D40028001D32200
:10FB8C00EFC394044011EFD39420500BEFF4045FB7
:09FB9C00B50702D322C322C322E3
:10FB5700EFC394024013EFD39410500DEFF4045FFA
:0BFB67006F6004EFB40C02D322C32235
:04E917007816E6FF89
:10E91B00EF12CCBFE95980E95C81E95F82E9628340
:10E92B00E96584E96885E96B88E96E89E9718AE9AB
:10E93B00748BE9778CE97A8DE97D90E98091E98395
:10E94B0092E98693E98994E98C950000E98F7F1B06
:10E95B00227F82227F37227F38227F39227F8422B7
:10E96B007F81227F83227F34227F35227F36227F55
:10E97B0085227F2A227F30227F31227F32227F33F2
:07E98B00227F0D227FFF2215
:10FBEC0012E91BC3EF648094B04008D3EF64809497
:05FBFC00B94002E4FF26
:01FC010022E0
:10F5EA00E4F511C21C902285F0FFE50BFDEFFB3319
:10F5FA0095E0FAC3EB9D7480F86A985016EFFD33D4
:10F60A0095E0FC74882DF58274223CF5837401F030
:03F61A000F80D787
:01F61D0022CA
:05F7B20090229AEFF027
:10F7B700C21A7B017A20790012FB72EF7014D21AF9
:10F7C700C21C7B017A20790012EDCC90229AE0F8D6
:04F7D700A607A21AC5
:01F7DB00220B
:10804E00E50C12CCBF80C900811201812E02900274
:10805E000382E104833B0583800683B5078402080F
:10806E00823709820B0A821E0B85930C85D90D86E9
:10807E00260E8DE50F8F1F108F9A118B4A128C01D1
:10808E001387D014880F1588DA168910178952189D
:10809E0089A41989DA1A8A1D1B8A751C8AC41D8C3B
:1080AE00591E8D001F872B2086832186E92286B8D4
:1080BE002386D5248E9825000090FD12926E7ACDDF
:1080CE0079841291617ACD799612FAA57B007A00A5
:1080DE00791312FAA57BFF7ACD799C12FAA57B0053
:1080EE007A00790E12FAA57BFF300C067ACD799EB6
:1080FE0080047ACD79A512FAA5788C761708767059
:10810E00750C01227F1612F7B250087816E660033E
:10811E00750C02788DE618466003029100028623E4
:10812E001291931293FD12E235FFE511C39F504059
:10813E0012E2BA0412937B129405400E12E2BA2494
:10814E000312937B2404FF12F3711292967ACD7967
:10815E00B212FAA512E2BA246C1292F2246D1293A4
:10816E0060407112E2BA246E1292F2246F0281DB29
:10817E0012E23512E28904FF12F37112E23512E2B5
:10818E0089129405401812E23512E2892403FF1277
:10819E00F37112E23512E2892404FF12F371129286
:1081AE00967ACD79B812FAA512E23512E289245CDC
:1081BE0012928612E29A245D129360401712E235F3
:1081CE0012E29A245E12928612E29A245FF8E60474
:1081DE00FF12F371300C0C051112E23512E26740FA
:1081EE0011800C051112E235FFE511C39F4003E427
:1081FE00F511788C760B0876B8750C032212E27E98
:10820E00FF12FCCE40201291707ACD79BE028CD432
:10821E0012E22B782526FF12FCC3400A1291707AC7
:10822E00CD79CC028CD40286CE7BFF7ACD79DA1250
:10823E00FAA5E512640360030282DB12E2272F2403
:10824E005BF8E604FF12F3711292D37ACD79E11244
:10825E00FAA530122312E2272F243BF8E6547F783A
:10826E0017F6C3940A500512939B802F12E2C94051
:10827E003012932324F6802312E2272F243BF8E6B4
:10828E00541F7817F6C39405500512936D800C1287
:10829E00E2D0400D12932324FB25E0FF12F37180F0
:1082AE00031293B07BFF7ACD79EC12FAA512E22776
:1082BE002F243BF8E67BFF30E7067ACD79F0800479
:1082CE007ACD79F512FAA5750C08028605750C069D
:1082DE00028605788DE618467003750C027F16121D
:1082EE00F7B2400302910012E21B600912E213750D
:1082FE000C050286A2300C0C12E917EF6484700490
:10830E000512800D300C1812E917EF6485701015E8
:10831E001253120312E2131293467D05028F871237
:10832E00E917EF641B6003029100028623788DE645
:10833E0018467003750C027F1612F7B240030291B5
:10834E000012E21B600912E21312E2D70287081232
:10835E00E917EF640D600612E917BF830712E209F1
:10836E0012E2D72212E917EF641B6003029100029A
:10837E008623788DE618467003750C027F1612F769
:10838E00B2400302910012E21B600E12E213750C52
:10839E000712E29378260289FE12E917EF641B603A
:1083AE0003029100028623788DE618467003750C41
:1083BE00027F1612F7B2400302910012E21B600C0C
:1083CE00E6FF24D07827F612FCEE801112E917BFD3
:1083DE000D147826E67827F6782612E21190229868
:1083EE00740CF0028FF012E917EF641B6003029118
:1083FE0000028623788DE618467003750C027F16F0
:10840E0012F7B2400302910012E21B6038E66430AC
:10841E00701912E22B12E2E1446012930D7ACD79BB
:10842E00F012FAA530141BD20D801712E22B12E2B5
:10843E00E1444012930D7ACD79F512FAA53014026B
:10844E00D20D02860512E917EF648470763012346D
:10845E0012E255547F7817F6700302857316129246
:10846E001912E23E301402D20D12932CC3940A500C
:10847E000612939B0284C412E2C940411293A724B0
:10848E00F60284C412E255541F7817F67003028563
:10849E0073161291CE12E23E301402D20D12932CAC
:1084AE00C39405500512936D800C12E2D0400E124B
:1084BE0093A724FB25E0FF12F3710285731293B08C
:1084CE0002857312E917EF6485600302857D301211
:1084DE004412E255547F7817F6C3945A400302852E
:1084EE00730612921912E23E301402D20D1293D17B
:1084FE00C3940A500E7F2B12FCEEC3740A781796A3
:10850E0002856412E2C940547F2D12FCEE7817E604
:10851E0024F602856412E255541F7817F6C3941F91
:10852E005043061291CE12E23E301402D20D129337
:10853E00D1C39405500F7F2B12FCEEC37405781730
:10854E009625E0801112E2D040127F2D12FCEE78BB
:10855E0017E624FB25E0FF12F37180097BFF7ACD2D
:10856E0079E712FAA57D107F0212FB3B028B7A127D
:10857E00E917EF641B600B12E917EF640D6003023D
:10858E009100028623E512701212E22B12E279128A
:10859E0093C2301434D203D201802EE512640170DE
:1085AE001012E22B12E2791293DC30141CD20380EB
:1085BE0018E5126402701212E22B12E2E1FB12E2D3
:1085CE007E1293E9301402D201804A788DE6184665
:1085DE007003750C027F1612F7B24003029100125F
:1085EE00E21B6016902284E014600304700912E20C
:1085FE002B12933712E2E8028B7A12E917BF0D0A9B
:10860E007824E6FF12DFE70289D712E917EF641B21
:10861E0060030291000289D7788DE61846700375C3
:10862E000C027F1612F7B2400302910012E21B6099
:10863E0016902284E014600304700912E22B129348
:10864E003712E2E8028B7A12E917BF0D1A7824E688
:10865E00FF12D0B612E672750C02201403029100BE
:10866E00D203D201D20E2212E917EF641B6003026D
:10867E0091000289D7788DE618467003750C027F3B
:10868E001612F7B2400302910012E21B600E12E2C4
:10869E0013750C2212E29378240289FE12E917EF69
:1086AE00641B60030291000289D712E22B78252603
:1086BE00FF12FCF8400A1291A07ACD79FA028CD4FE
:1086CE00902298E0F50C2212E22B782526F508FF71
:1086DE0012F896301402D20A0289D7788DE618461F
:1086EE007003750C027F1612F7B24003029100124E
:1086FE00E21B600E12E21312E2EF12E293782502F1
:10870E0089FE12E917BF0D0712E20912E2EF2212DB
:10871E00E917EF641B60030291000289D7788DE69A
:10872E0018467003750C027F1612F7B240030291C1
:10873E000012E917BF1B03750C0212E917BF0D19C2
:10874E007824E6FF6010C374049FFF12F84E12EBFC
:10875E00C3301402D20F0289D712E21B70030291AA
:10876E000074D026F6E66401701312E21312926EB4
:10877E007ACE79071291611293867824F67817E6ED
:10878E006402701312E2131292A07ACE792912911A
:10879E00841293867824F67817E66403700D12918E
:1087AE00017ACE794B1293F67824F67817E66404A4
:1087BE0060030291001291017ACE795C1293F60257
:1087CE008E31788DE618467003750C027F1612F7FF
:1087DE00B2400302910012E917BF1B030289D712A0
:1087EE00E917EF640D60030291001292A07ACE7920
:1087FE006D1291847ACE797D12FAA5750C15028BC5
:10880E007A788DE618467003750C027F1612F7B251
:10881E00400302910012E917BF1B030289D712E928
:10882E0017EF648170141291937ACE798E1291B4EF
:10883E007ACE799F12FAA5028B7A12E21B7003028E
:10884E009100E6B4311012E213750C161291C17A32
:10885E00CE79B012FAA57817E6B4321012E213757B
:10886E000C191291C17ACE79BF12FAA57817E66467
:10887E0033702712E213750C1C12920C300C0D7A09
:10888E00CE79CE1291B47ACE79DF800B7ACE79F092
:10889E001291FF7ACF790112FAA57817E664346047
:1088AE000302910012E213750C1D12920C30120E7F
:1088BE007ACF79121291FF7ACF7922028CD47ACFA5
:1088CE0079331292467ACF7943028CD4788DE6189A
:1088DE00467003750C027F1612F7B2400302910028
:1088EE0012E21B600F12E213750C1712E29378243A
:1088FE00F612FCEE12E917EF641B60030291000200
:10890E0089D7788DE618467003750C027F1612F71C
:10891E00B2400302910012E21B600E12E213750CBC
:10892E001812E29378250289FE12E917BF0D07127D
:10893E00E209750C182212E917EF641B600302910D
:10894E00000289D712E22B782526FF12FB8C400AF3
:10895E001291A07ACF7954028CD4129253F50D1243
:10896E00E898E50D75F00A842430F513E50D75F0E1
:10897E000A84E5F02430F514E4F515FB7A0079133A
:10898E009022A812CC960B7A2279B112FA83AF0DEF
:10899E0012F902028A8F788DE618467003750C0262
:1089AE007F1612F7B2400302910012E21B600F1203
:1089BE00E213750C1A12E2937824F612FCEE12E909
:1089CE0017EF641B6003029100028A8F788DE61800
:1089DE00467003750C027F1612F7B2400302910027
:1089EE0012E21B600F12E213750C1B12E293782534
:1089FE00F6028FCE12E917BF0D0712E209750C1B96
:108A0E002212E917EF641B6003029100028A8F1293
:108A1E00E22B782526FF12FB57401012E2C1750C8F
:108A2E00011292D37ACF7974028CD4129253F50B31
:108A3E0012E898E50B75F00A842430F50EE50B75F7
:108A4E00F00A84E5F02430F50FE4F510FB7A007996
:108A5E000E9022A812CC960B7A2279AE12FA83AF20
:108A6E000B12F8DE028B64788DE618467003750CD7
:108A7E00027F1612F7B2400302910012E917BF1BD4
:108A8E0003028B6412E21B7003029100E6B43110F4
:108A9E00D20CA20CE433FF12F92612E213750C026B
:108AAE007817E664326003029100C20CA20C33FF09
:108ABE0012F926028B44788DE618467003750C0267
:108ACE007F1612F7B2400302910012E917BF1B0383
:108ADE00028B6412E21B7003029100E6643170296E
:108AEE00902299F0902299E0FFC39410500B743CA1
:108AFE002FF8760AE004F080EBD212A212E433FFD4
:108B0E0012F96E12E213750C027817E664326003E6
:108B1E00029100902299F0902299E0FFC394105098
:108B2E000B743C2FF87605E004F080EBC212A21213
:108B3E00E433FF12F96E12E2130290FD788DE618FF
:108B4E00467003750C027F1612F7B24003029100B5
:108B5E0012E917BF1B030290FD12E917BF81111214
:108B6E0092797ACF798412FAA5750C1312E2132238
:108B7E0012E21B7003029100E66431704A12E21396
:108B8E00750C201292E712F8727818EFF67009122F
:108B9E0091257ACF799580287818E6B4010912913B
:108BAE00257ACF79A680197818E67BFFB402067A6B
:108BBE00CF79B780047ACF79C81292467ACE7918D7
:108BCE0012FAA5E47824F67817E66432600302916F
:108BDE000012E213750C211292797ACF79D912FA1A
:108BEE00A5AF0812F3717BFF7ACF79DB12FAA5E4F9
:108BFE00028E31788DE618467003750C027F1612C0
:108C0E00F7B2400302910012E917BF1B030290FD59
:108C1E0012E21B7003029100E664336003029100BE
:108C2E0012E213750C1E902284F01292AB7ACF7959
:108C3E00DE12FAA57D041293BA7ACF79EA12FAA55A
:108C4E007D047F0212FB3BE4028E31788DE61846DE
:108C5E007003750C027F1612F7B2400302910012D8
:108C6E00E9177817EFF624F3600724F2705B029091
:108C7E00FD7824E6FFD394004040EFD3950B503A95
:108C8E0016E62488F582E43422F583E06401700947
:108C9E00750C1F12E213028D7412E21312FD3E7D4B
:108CAE00017F0112FB3B7BFF7AD0790812FAA57D7A
:108CBE00011293BA7AD07916800C1292E712E2C1A1
:108CCE007BFF7ACD79CC02FAA512E21B70030291DA
:108CDE0000902284E014600604600302910012E208
:108CEE001312E22BFE7817E6FF2E24D07824F6021C
:108CFE008DDE788DE618467003750C027F1612F71E
:108D0E00B2400302910012E9177817EFF624F360D0
:108D1E000724F2707C0290FD902284E0D3940040F0
:108D2E003AD3902283E094FF902282E09400400692
:108D3E00E4F0A374FFF0902283E0FF7824E6FE2493
:108D4E008EF8A607748E2EF8E6FF74572EF582E481
:108D5E003421F583EFF0301402D20E750C1F12E29F
:108D6E0013E4902284F01292AB7ACF79EC12FAA52A
:108D7E007824E6248EF8E6FF12EAF71292DD7ACF17
:108D8E0079FA12FAA5E4902284F0902282F0A3F0F0
:108D9E002212E21B7003029100902284E024FD5007
:108DAE000302910012E213902282E0FEA3E0FF7C08
:108DBE00007D0A12C97C7817E6F97A002FFDEA3E8B
:108DCE00CD24D0FEED34FF902282F0A3CEF0AF0181
:108DDE0012FCEE12E2E822788DE618467003750C4E
:108DEE00027F1612F7B2400302910012E917BF82FA
:108DFE0017750C0D1293007AD0792012FAA512E293
:108E0E0013E4902284F0801B12E917BF8319750CAE
:108E1E000E1293007AD0792E12FAA512E213E49074
:108E2E002284F07824F62212E21B601A12E2131248
:108E3E00E2A61292B81293917AD0793D12FAA578E1
:108E4E0017E6FF028FCE300C3312E917EF64846001
:108E5E000812E917EF64857023E4F51212E213FD90
:108E6E007F0212FB3B7BFF7AD0797E12FAA512931A
:108E7E00917AD0793D12FAA5750C102212E917EFEE
:108E8E00641B60030291000290FD12E2C1750C0199
:108E9E00E51270247817F67817E6C3950B500E126C
:108EAE00E2297825261293C278170680EA20140349
:108EBE00029100D203D20122E512640170237817C9
:108ECE00F67817E6FFC3950B500E12E22B78252687
:108EDE001293DC78170680E9201403029100D20366
:108EEE0022E512640260030291007817F67817E605
:108EFE00FFC3950B5012EF541FFB12E22B78252661
:108F0E001293E978170680E5201403029100D2012E
:108F1E0022788DE618467003750C027F1612F7B292
:108F2E00400302910012E21B601412E21312E2A639
:108F3E007D0C7F0112FB3B7817E6FF028FCE12E904
:108F4E0017EF648470160512E512C394034003E410
:108F5E00F51212E2131292B87D0C801D12E917EF72
:108F6E006485701A1512E512C3940340037512023C
:108F7E0012E213E41293467D0C7F0102FB3B12E9D1
:108F8E0017EF641B60030291000290FD788DE618C6
:108F9E00467003750C027F1612F7B2400302910061
:108FAE0012E21B601E9022987425F0750C0AE6FFE3
:108FBE0024D0FE7825F67824E67826F67827A606BD
:108FCE0002FCEE12E917BF0D1D7824E67825F6FF98
:108FDE00E47824F69022987425F0E47826F6782723
:108FEE00A607750C0A2212E917EF641B60030291A3
:108FFE00000290FD7F1612F7B240030290F412E9C0
:10900E00177817EFF6247F60301470030290B524A2
:10901E00FE6045146045245B60030290CC129411EF
:10902E007F2A12FCEE750C0F12E213300C047F0037
:10903E0080027F018F120290F41294117BFF7AD07E
:10904E00794A12FAA51292DD7AD0795B12FAA575D9
:10905E000C1212E2130290F40290AF300C1112E2D5
:10906E003312E267401812E2B225E0F511800F12BA
:10907E00E233FFE511C39F400512E2B2F511300C49
:10908E001112E23312E267401812E2B225E0F51136
:10909E00800F12E233FFE511C39F400512E2B2F5D5
:1090AE0011750C020290F412E213750C04300C04CC
:1090BE007F0080027F011291381293FD802812E208
:1090CE001B602312E213750C0512E2A9300C047F0B
:1090DE000080027F011291387ACD79AC12FAA57810
:1090EE0017E6FF12FCEE788DE618467005800075C7
:0290FE000C0262
:1091000022788C762708761012FD3EE4FD7F01124E
:10911000FB3B7BFF7ACE793A12FAA5E4FD7F02127F
:10912000FB3B7BFF227BFF7ACE793A12FAA5E4FD66
:109130007F0212FB3B7BFF228F1212FD3EE4FD7F7C
:109140000212FB3BE51275F00EA4247EF974D035B3
:10915000F0FA7BFF12FAA5E4FD7F0112FB3B7BFFD7
:10916000227BFF12FAA5E4FD7F0212FB3B7BFF226C
:10917000788C760F0876A0750C01E4FD7F0212FB57
:109180003B7BFF227BFF12FAA5E4FD7F0212FB3B33
:109190007BFF2212FD3EE4FD7F0112FB3B7BFF22A1
:1091A000788C760F0876A0750C01E4FD7F0212FB27
:1091B0003B7BFF2212FAA5E4FD7F0212FB3B7BFF03
:1091C0002212FD3EE4FD7F0112FB3B7BFF22EE7588
:1091D000F00AA42F14541F4420FBE6547F9022A9C8
:1091E000F0E4FD7FFF12D7F87817E625E0FFC3749F
:1091F0005A9FFF7825E6FE7824E675F00AA422122D
:10920000FAA5E4FD7F0212FB3B7BFF2212FD3EE448
:10921000FD7F0112FB3B7BFF22EE75F00AA42F14A9
:10922000541F4420FBE6547F9022A9F0E4FD7FFF09
:1092300012D7F8C3745A781796FF7825E6FE78247B
:10924000E675F00AA42212FAA5E4FD7F0212FB3BA8
:109250007BFF22E4FD7F0212FB3B7BFF7ACF796329
:1092600012FAA57824E675F00AA47825262212FDC4
:109270003EE4FD7F0112FB3B2212FD3EE4FD7F0137
:1092800012FB3B7BFF22F8E604FF12F371E50B248F
:10929000031313543F22E4FD7F0212FB3B7BFF22AA
:1092A00012FD3EE4FD7F0112FB3B2212FD3EE4FD78
:1092B0007F0112FB3B7BFF22E4FD7F0212FB3BE5BB
:1092C0001275F00EA4247EF974D035F0FA7BFF12EB
:1092D000FAA522E4FD7F0212FB3B7BFF22E4FD7F27
:1092E0000212FB3B7BFF2212FD3EE4FD7F0112FBDD
:1092F0003B22F8E604FF12F371E51125E025E02298
:1093000012FD3EE4FD7F0112FB3B7BFF22FBE4905C
:1093100022A9F0FD7FFF12D7F87D0C7F0212FB3BE4
:109320007BFF227F2D12FCEE7817E6227D057F025F
:1093300012FB3B7817E622FE7817E6FF2E24D07842
:1093400024F612FCEE22FD7F0212FB3BE51275F0C3
:109350000EA4247EF974D035F0FA7BFF12FAA52210
:10936000F8E604FF12F371E50BD39402227F2B126F
:10937000FCEEC3740578179625E022FF12F371E521
:109380001125E025E0227ACE791812FAA57817E6A1
:1093900022E4FD7F0112FB3B7BFF227F2B12FCEEC0
:1093A000C3740A781796227F2D12FCEE7817E622F6
:1093B0007BFF7ACD79E712FAA5227F0212FB3B7B75
:1093C000FF2214FDEF541FFB9022A9EDF012D7F8F5
:1093D000227D057F0212FB3B7817E62214FDE49004
:1093E00022A9F07BFF12D7F822149022A9F0E4FD05
:1093F0007FFF12D7F82212FAA57817E6227ACD79E4
:10940000AC12FAA5222402FF12F371E50BD39402E9
:0C9410002212FD3EE4FD7F0112FB3B2216
:10F2F300496E697469616C697A696E6700506C65FF
:10F3030061736520776169742E2E2E202000436F70
:10F313006E74696E75653A20456E7465720043615B
:0FF323006E63656C3A2020204573632020200024
:10E8170043D002782876070876D012FC0212FC70E3
:10E8270012FAE412F33212F1EFD2AF12F09F12FD97
:10E837003EE4FD7F0112FB3B7BFF7AF279F312FA8C
:10E84700A5E4FD7F0212FB3B7BFF7AF3790012FA06
:10E85700A512D5BA12800612E67212FD4F12F5EA1A
:10E8670012F64F12F61E90280774FFF012804EE43E
:10E87700902807F012941C12A59712E2F912F57D61
:10E8870012DA0712B49A12C38612F05A12FC2B80BE
:01E89700D2AE
:10FC700090280974FFF0902807F0E4902805F022FE
:10FAE400902814E054FBF0902816E04480F090280D
:0DFAF40014E04480F0902812E0547FF022CE
:10F05A00C2C712FCE4D2C7EF642370389028077441
:10F06A00FFF012FD3EE4FD7F0112FB3B7BFF7AF3CA
:10F07A00791112FAA5E4FD7F0212FB3B7BFF7AF3BA
:10F08A00792112FAA5E4902807F0750C14788C7689
:04F09A0027087610BD
:01F09E00224F
:08F7F4004122810041225D0069
:10DE8600902299E0FF04F0745E2FF582E43422F5C7
:10DE960083E022902299E0FF12F5B490229CEFF0E5
:10DEA6002290229CE0FF90229AE02458F582E434E6
:10DEB60022F583EFF0902299E004F022902299E077
:10DEC600FF12F5B490229DEFF090229CE014F0E052
:10DED600C3950B2290229CE075F00AA4F09022993B
:10DEE600E0245E22902299E0FF12F5B490229DEF85
:10DEF600F090229CE014F0A3E014F090229CE0C382
:10DF060022E075F06484E5F075F00A842430FF227F
:10DF160024D0FF90229CE02FF090229BE004F0E0BA
:10DF26002290229AE0FF2458F582E43422F583E019
:10DF3600FE22E075F00A84E5F0243022902257E0B4
:10DF4600FF902299E0D39F2290225EE064522290B5
:10DF5600225EE0645322F583EEF090229AE004F00C
:10DF6600E02290225EE0644122E075F06484243071
:10DF7600FF2290225EE0644722A3E004F0E0C3940F
:10DF86000422902299E0FF12F5B490229DEFF02230
:10DF9600E0FEA3E0FF7C007D0A02C97C90225EE0E1
:10DFA60064432290225EE0644522E490229BF0A323
:10DFB600F02290229BE0D39403227F0212F5B4EF65
:10DFC600FD7C0022EE9390229CF0C3944122243DD6
:10DFD600F582E43421F5832212CC2190229F02CCD3
:01DFE6002D0D
:06F545009022A512CC96F5
:10F54B00E49022A8F09022A512CC7612800E902285
:10F55B00A8E0FEC39F501A9022A512CC768E82751E
:10F56B00830012C91BFF12FBA59022A8E004F080B8
:01F57B00D4BB
:01F57C00226C
:10F5B400E4FD12DE8DFC642C6029902257E0FBEF01
:10F5C400C39B40037FFF22EC24D0FED39409400365
:10F5D4007FFF22ED75F00A84E5F075F00AA42EFD94
:05F5E4000F80CFAF0510
:01F5E90022FF
:02ECD500AA078C
:10ECD700E49022A5F0A3F0745E2A12DE90FE642C65
:10ECE700602E902257E0FFEAC39F40037FFF22EE8A
:10ECF70024D0FBD3940940037F00229022A512DF82
:10ED070096EB2FFFEC3E9022A5F0A3EFF00A80C709
:10ED17009022A5E060099022A5E4F0A374FFF0908B
:04ED270022A6E0FF41
:01ED2B0022C5
:05F7050012F829921A20
:10F70A00902257E0C39403500122902260E0B42C67
:10F71A0002D32212DFC0BC0205BD5502D322EF6517
:06F72A00086002D322C3B7
:01F7300022B6
:10F82900902257E0C39403500122902260E0B42C47
:10F8390002D32212DFC0BC0205BD5502D322EF60FC
:04F8490002D322C301
:01F84D002298
:0AFD02007F3F12FBA57F0D02FBA559
:0AFD0C007F2A12FBA57F0D02FBA564
:10F9B6009022A5EFF0D39463400612DF6F12FBA5E9
:10F9C6009022A512DF0712FBA59022A512DF38FFB1
:03F9D60002FBA58C
:10FAC6009022A5EFF012DF7012FBA59022A512DF9F
:0EFAD6000712FBA59022A512DF38FF02FBA548
:10A5970020050302B2A8C20590225EE0B4521FA3B1
:10A5A700E0B4551A12F70A500302B2A312FD0CAF1A
:10A5B7000D12F9B67F2C12FBA5AF0B02A7B212DF63
:10A5C7004E7004A3E06453701F12F7055006301A4B
:10A5D7000302B2A3301A0312FD0C301405D2020293
:10A5E700B2A312000002B2A312DF4E7004A3E0640C
:10A5F7004F702A12F70A500302B2A3E4902299F08F
:10A6070012DE86B42CFA12DE9912DED2400302B2B1
:10A61700A012B470246CF8E604FF02A7B212DF7828
:10A627007004A3E0644F703412F70A500302B2A318
:10A63700E4902299F012DE86B42CFA12DE9912DE2B
:10A64700D2400302B2A012FD0C12B39D12B3F290D6
:10A65700229CE0246CF8E604FF02A7B2300C4612F5
:10A66700DF787004A3E06441703B12F70A500302DD
:10A67700B2A3E4902299F012DE86B42CFA12DE9986
:10A6870012DED2400302B2A012FD0C7F6112FBA5BD
:10A697007F6F12B42712B3F290229CE0245CF8E695
:10A6A70004FF02A7B212DF787004A3E0644D703C88
:10A6B70012F70A500302B2A3E4902299F012DE8641
:10A6C700B42CFA12DE99600302B2A012FD0CE490DA
:10A6D700229EF090229EE0C3950B400302B2A31284
:10A6E700B39D12B401246C12B44780E712DF557092
:10A6F70004A3E06453702E12F70A500302B2A3E4D6
:10A70700902299F012DE86B42CFA12DE997004C2F8
:10A7170018800990229CE0B40108D21812FD0C029F
:10A72700B18202B2A0300C4E12DF787004A3E0644D
:10A7370042704312F70A500302B2A3E4902299F041
:10A7470012DE86B42CFA12DE99600302B2A012FD63
:10A757000CE490229EF090229EE0C3950B400302EA
:10A76700B2A37F6712FBA57F6112B42712B401243D
:10A777005C12B44780E0300C3812DF687004A3E045
:10A78700644F702D12F70A500302B2A3E490229986
:10A79700F012DE86B42CFA12DE9912DED2400302E2
:10A7A700B2A012B470245CF8E604FF12F9B602B145
:10A7B7008212DF4E7004A3E06443704E12F7055017
:10A7C70006301A0302B2A3E4902299F012DE86B48F
:10A7D7002CFA12DE99D394634009201A0302B2A31C
:10A7E70002B2A0301A0812B2CD7F0D12FBA590223B
:10A7F7009CE0FF12D0B612E67220140302B2A3D275
:10A8070003D201D20DD20E02B2A312DFA27004A3AB
:10A81700E06443703D12F7055006301A0302B2A3F5
:10A82700E4902299F012DE86B42CFA12DE99D394C2
:10A83700634009201A0302B2A302B2A0301A081219
:10A84700B2CD7F0D12FBA590229CE0FF12DFE7023D
:10A85700B2A312DF4E7004A3E06456600302A8FCA3
:10A8670012F70A500302B2A312B45A7AE6793212E7
:10A87700B463502190E63212DFCA400AE0FF945BCE
:10A887005004EF4420F090229CE0FF600312FBA5E8
:10A8970012DEBB80D6E4902299F07AE6794F12B4A3
:10A8A70063502190E64F12DFCA400AE0FF945B50E5
:10A8B70004EF4420F090229CE0FF600312FBA512F6
:10A8C700DEBB80D67BFF7AE6796012F5457B017A9D
:10A8D7002279B112F5457BFF7AE6796612F5457B59
:10A8E700017A2279AE12F5457BFF7AE6796F12F588
:10A8F70045E402AF4412DFA27004A3E06442704D46
:10A9070012F829500302B2A3E4902299F012DE86CE
:10A91700B42CFA12DE99BF60047F03801F90229C3B
:10A92700E0B430047F02801490229CE0B418047FC6
:10A9370001800990229CE0B40C08E4FF12F84E1243
:10A94700EBC320140302B2A3D20F02B2A312DFA2F9
:10A957007004A3E06441704612F70A500302B2A3E1
:10A96700E4902299F012DE86B42CFA12DE99E014F4
:10A97700F0E0C3950D400302B2A012B45A90229999
:10A98700E0FFC3950B500C90229CE012B47812DEC6
:10A99700BB80EA20140302B2A3D20302B2A3300C95
:10A9A7005312DF687004A3E06441704812F70A503D
:10A9B7000302B2A3E4902299F012DE86B42CFA12B5
:10A9C700DE99E014F0E0C3950D400302B2A012FD3A
:10A9D7000CE4902299F0902299E0FFC3950B50095F
:10A9E700EF12B41412DEBB80ED20140302B2A3D21F
:10A9F7000102B2A312DFA27004A3E06453705012E5
:10AA0700F70A500302B2A3E4902299F012DE86B44B
:10AA17002CFA12DE99E4902299F012DE86B42CFA11
:10AA270012DE86642C600612DF4240F42212DEEA50
:10AA3700950D5007A3E0C3950B400302B2A012B4D3
:10AA47003A12B47820140302B2A3D20302B2A3309D
:10AA57000C5B12DF687004A3E06453705012F70AAE
:10AA6700500302B2A3E4902299F012DE86B42CFAC6
:10AA770012DE99E4902299F012DE86B42CFA12DEE7
:10AA870086642C600612DF4240F42212DEEA950D3E
:10AA97005007A3E0C3950B400302B2A012B484127F
:10AAA700B41420140302B2A3D20102B2A3300C7370
:10AAB70012DF687004A3E0644D706812F70A500350
:10AAC70002B2A3E4902299F012DE86B42CFA12DEC9
:10AAD70099E4902299F012DE86B42CFA12DE86648D
:10AAE7002C600612DF4240F42212DEC25007A3E0B8
:10AAF700C39402400302B2A012B48490229C600760
:10AB0700E0541F44608005E0541F4440FBE490225A
:10AB1700A9F0FD7FFF12D7F820140302B2A3D20DCC
:10AB270002B2A3200C0302ABD712DF687004A3E0C4
:10AB37006456600302ABD712F70A500302B2A3E4CC
:10AB4700902299F012DE86B42CFA12DE99E4902254
:10AB570099F012DE86B42CFA12DE86642C60061297
:10AB6700DF4240F42212DEC25007A3E0C3946440E0
:10AB77000302B2A012B43AFE12DFD4EFF03014028F
:10AB8700D20DEFC3945A400690229D745AF03012AA
:10AB970011EE541F4420FB90229DE0FFC3745A9F7F
:10ABA700801E90229DE0C3941C5003741CF09022D9
:10ABB7009CE0541F4420FBA3E0FFC3745A9FC313B8
:10ABC700547F9022A9F0E4FD7FFF12D7F802B2A3C9
:10ABD700300C5912DF687004A3E06452704E12F70C
:10ABE7000A500302B2A3E4902299F012DE86B42C35
:10ABF700FA12DE9912DED2400302B2A012FD0C7FD8
:10AC07003012FBA590229CE0243CF8E630E7047F55
:10AC17003180027F3012FBA57F2C12FBA590229C6E
:10AC2700E012DFD4E0FF12F9B602B18212DFA97099
:10AC370004A3E06441600302ACBE12F70A500302AA
:10AC4700B2A3E4902299F012DE86B42CFAE49022A3
:10AC57009AF012DFB012DEE312DE90FF642E602856
:10AC6700EF642C602312DEDA12DE9012DF16B403D3
:10AC77000AA3E0D394FF400302AD9C12DFB8400360
:10AC870002AD9C12DEBB80CD12DEA712DF7F40C271
:10AC9700E490229AF012DF2774AB2FF582E4342177
:10ACA70012DF5CB404EF12FD0C12F3EB2014030265
:10ACB700B2A3D21502B2A312DFA97004A3E0644DB8
:10ACC700600302AD4912F70A500302B2A3E49022CF
:10ACD70099F012DE86B42CFAE490229AF012DFB0D3
:10ACE70012DEE312DE90FF642E6028EF642C6023EF
:10ACF70012DEDA12DE9012DF16B4030AA3E0D39451
:10AD0700FF400302AD9C12DFB8400302AD9C12DE88
:10AD1700BB80CD12DEA712DF7F40C2E490229AF0FB
:10AD270012DF2774512FF582E4342112DF5CB4045B
:10AD3700EF12FD0C12F45F20140302B2A3D2170224
:10AD4700B2A312DFA97004A3E06447600302ADD683
:10AD570012F70A500302B2A3E4902299F012DE869A
:10AD6700B42CFAE490229AF012DFB012DEE312DE7E
:10AD770090FF642E602AEF642C602512DEDA12DE63
:10AD87009012DF16B40309A3E0D394FF40028005B5
:10AD970012DFB8400612FD0202B2A312DEBB80CB5F
:10ADA70012DEA712DF7F40C0E490229AF012DF275D
:10ADB70074C02FF582E4342112DF5CB404EF12FD76
:10ADC7000C12F49920140302B2A3D21602B2A312F2
:10ADD700DFA97004A3E06454600302AED712F70A38
:05ADE700500302B2A3BD
:10ADEC00E4902299F09022A3F0A3F012DE86B42C0A
:10ADFC00FA12DEE3F9E43422FA7B0190227E12CCC3
:10AE0C009612DEE312DE90FFC394304030EFD39401
:10AE1C0039502A902299E0FBC3941050209022A321
:10AE2C0012DF96745E2B12DE902FFFEC3ECF24D0F7
:10AE3C00CF34FF9022A3F0A312DEB980C412DEE35C
:10AE4C00F582E43422F583E4F09022A3E0FEA3E043
:10AE5C00FF643C4E604CEF642C7003EE6401604266
:10AE6C00EF64587003EE64026038EF64847003EE94
:10AE7C006403602EEF64087003EE64076024EF64D3
:10AE8C00107003EE640E601AEF64207003EE641C05
:10AE9C006010EF64507003EE64466006BE7029BF0C
:10AEAC00802690227E12CC769022A812CC967B0122
:10AEBC007A21792C12FA8312FD0C12F1262014033C
:08AECC0002B2A3D20002B2A3FE
:10AED40002B2A012DF4E7004A3E06441706912F75D
:10AEE4000A500302B2A312FD0C9021AB12B32190BD
:10AEF40021AB12B2A99021AB12B3137F2E12FBA582
:10AF04009021AC12B3219021AC12B2A99021AC12C1
:10AF1400B3137F2E12FBA59021AD12B32D9021AD5A
:10AF240012B2BB9021AD12B3397F2E12FBA5902132
:10AF3400AE12B32D9021AE12B2BB9021AE12DF3807
:10AF4400FF12FBA502B18212DF4E7004A3E0644D30
:10AF5400706212F70A500302B2A312FD0C90215141
:10AF640012B35990215112B2EF90215112B3397F8B
:10AF74002E12FBA590215212B35990215212B2EF16
:10AF840090215212B38F7F2E12FBA590215312B33E
:10AF9400B790215312B30190215312B38F7F2E1215
:10AFA400FBA590215412B3B790215412B301902100
:10AFB4005402B02612DF4E7004A3E06447706D1291
:10AFC400F70A500302B2A312FD0C9021C012B3D1B0
:10AFD4009021C012B3479021C012B3C37F2E12FB3D
:10AFE400A59021C112B3D19021C112B3479021C1C0
:10AFF40012B3C37F2E12B48C12DF6F12B48C12DF23
:10B004000712FBA59021C212DF38FF12FBA57F2E89
:10B0140012B49312DF6F12B49312DF0712FBA590E0
:10B0240021C312DF38FF12FBA502B18290225EE039
:10B03400B4521CA3E0B4541712F70A500302B2A38B
:10B0440012FD0C7B017A21792C12F54502B1821292
:10B05400DF557004A3E06473706612F70A500302AC
:10B06400B2A3E4902299F012DE86B42CFA12DE998F
:10B07400E4902299F012DE86B42CFA12DE86B42C07
:10B08400FA902299E0FF12ECD512DECA400302B214
:10B09400A012FD0C90229DE0FF90229CE0FE248EE5
:10B0A400F8A607748E2EF8E6FF74572EF582E43462
:10B0B40021F583EFF020140302B2A3D20E02B2A34F
:10B0C40012DF787004A3E06473703012F70A50033F
:10B0D40002B2A3E4902299F012DE86B42CFA12DEB6
:10B0E4009912DED2400302B2A012FD0C90229CE021
:10B0F400248EF8E6FF12FAC602B18212DF557004FC
:10B10400A3E06478600302B18A12F70A500302B222
:10B11400A3E4902299F012DE86B42CFA12DE99127E
:10B12400DED2400302B2A012FD0C90229F12CC4545
:10B1340000000001E4902299F0902299E0C3950D5B
:10B14400503C90229CE025E025E02468F582E4341C
:10B1540021F58312DFDE12CBB6EC4D4E4F60047F37
:10B164007880027F6F12FBA590229F12CC21780178
:10B1740012CC0E90229F12CC3912DEBB80BB7F0D05
:10B1840012FBA502B2A312DF557004A3E064617040
:10B194002B12F70A500302B2A3E4902299F012DEB4
:10B1A40086B42CFA12DE9912DED2400302B2A01247
:10B1B400B3DD12CC45FFFFFFFF02B2A312DF5570CF
:10B1C40004A3E06463702B12F70A500302B2A3E4F1
:10B1D400902299F012DE86B42CFA12DE9912DED295
:10B1E400400302B2A012B3DD12CC450000000002FD
:10B1F400B2A312DF557004A3E0642B704212F70A65
:10B20400500302B2A3E4902299F012DE86B42CFA21
:10B2140012DE99E014F012DE86B42CFA12DF8812E2
:10B22400DEFE950B5006A3E0950D400302B2A0127A
:10B23400B365C083C08212DFDE12CBC302B29212A6
:10B24400DF557004A3E0642D704D12F70A4050E4FA
:10B25400902299F012DE86B42CFA12DE99E014F0F2
:10B2640012DE86B42CFA12DF8812DEFE950B50062D
:10B27400A3E0950D4002802412B365C083C08212FE
:10B28400CC2D90229F12CC2112CBDD12CBB6D082D2
:10B29400D08312CC39800812F70A400312FD02E46D
:04B2A400902257F0AD
:10B2A80022E075F06484E5F075F00A842430FF121A
:10B2B800FBA522E075F06484E5F075F00A8424307B
:10B2C800FF12FBA52212FD0C90229CE075F00A8467
:10B2D8002430FF12FBA590229CE075F00A84E5F06B
:10B2E8002430FF12FBA522E075F06484E5F075F0C8
:10B2F8000A842430FF12FBA522E075F06484E5F08F
:10B3080075F00A842430FF12FBA522E075F00A8448
:10B31800E5F02430FF12FBA522E075F064842430A8
:10B32800FF12FBA522E075F064842430FF12FBA510
:10B3380022E075F00A84E5F02430FF12FBA522E034
:10B3480075F06484E5F075F00A842430FF12FBA5DB
:10B3580022E075F064842430FF12FBA52212FD0C54
:10B36800E47F01FEFDFC90229DE0F9F812CC0E90DE
:10B37800229F12CC3990229CE025E025E02468F534
:10B3880082E43421F58322E075F00A84E5F0243064
:10B39800FF12FBA5227F6712FBA57F6F12FBA57F1B
:10B3A8002012FBA5AF0812F9B67F2C12FBA522E0EC
:10B3B80075F064842430FF12FBA522E075F00A843E
:10B3C800E5F02430FF12FBA522E075F064842430F8
:10B3D800FF12FBA52212FD0C90229CE025E025E03F
:10B3E8002468F582E43421F5832290229CE004FF4E
:10B3F80012F9B67F3A12FBA52290229EE004FF12B2
:10B40800F9B67F3A12FBA590229EE022541FFB90CA
:10B41800229CE09022A9F0E4FD7FFF12D7F82212C7
:10B42800FBA57F2012FBA5AF0812F9B67F2C12FBF3
:10B43800A52212FD0C90229DE0FF90229CE022F8AC
:10B44800E604FF12F9B67F0D12FBA590229EE004D8
:10B45800F02212FD0CE4902299F0227BFF12800E5C
:10B46800902299E0FEC39F2212FD0C90229CE022BC
:10B47800FDE49022A9F07BFF12D7F82212FD0C9070
:10B48800229DE02212FBA59021C22212FBA5902149
:02B49800C322CD
:10E2F90020180302E397902257E0600302E3979006
:10E309002281E0FFC3950B5031744C2FF8E660224F
:10E319007F7012E39890228112E3B0902281E02469
:10E329004C12E3BC902281E0244CF8E4F6E004F0BE
:10E339008008902281E004F080C5902281E0850B5D
:10E34900F084E5F0F0300C4690225DE0FFC3950BB8
:10E359005031742C2FF8E660227F6112E3989022E5
:10E369005D12E3B090225DE0242C12E3BC90225DA3
:10E37900E0242CF8E4F6E004F0800890225DE00443
:10E38900F080C590225DE0850BF084E5F0F0221263
:10E39900FBA57F6312FBA57F2012FBA5AF0812F92D
:10E3A900B67F2C12FBA522E004FF12F9B67F3A12C0
:0FE3B900FBA522F8E6FF12F9B67F0D12FBA52295
:10EBC30012F8729022A5EFF0BF030B9022AA7425CE
:10EBD300F0A37480803B9022A5E0B4020B9022AA9C
:10EBE3007412F0A374C080299022A5E0B4010B90A5
:10EBF30022AA7409F0A3746080179022A5E09022E2
:10EC0300AA70087404F0A374B080067425F0A3748A
:0DEC130080F07F007E5A7D627C0212F2B319
:01EC200022D1
:10BE1F00496E76616C69642070617373776F7264B9
:10BE2F002100456E746572206E65772070617373A3
:10BE3F00776F72643A00456E746572206E65772075
:10BE4F0070617373776F726420616761696E3A0016
:10BE5F0050617373776F7264207375636365737367
:10BE6F0066756C6C79206368616E67656421004349
:10BE7F006F6D6D616E64204C6973743A004353208B
:10BE8F006E6E2C6D6D20202D20436F6E6E6563746A
:10BE9F0020766964656F20696E707574206E6E20F0
:10BEAF00746F206F7574707574206D6D0043412031
:10BEBF006E6E20202020202D20436F6E6E656374E0
:10BECF0020766964656F20696E707574206E6E20C0
:10BEDF00746F20616C6C206F757470757473005281
:10BEEF004F206E6E20202020202D2052656164206F
:10BEFF00636F6E6E656374696F6E20666F72206F0D
:10BF0F007574707574206E6E004343206E6E202022
:10BF1F002020202D2053617665206D617472697821
:10BF2F0020636F6E6E656374696F6E7320696E74D4
:10BF3F006F206D656D6F72792062616E6B206E6E12
:10BF4F00005243206E6E20202020202D205265733A
:10BF5F00746F7265206D617472697820636F6E6E95
:10BF6F00656374696F6E732066726F6D206D656D9A
:10BF7F006F72792062616E6B206E6E004342206E8D
:10BF8F006E20202020202D204368616E676520627F
:10BF9F006175642072617465206F6E2073657269BC
:10BFAF00616C206C696E652C0020202020202020E1
:10BFBF00202020202020206E6E3D31322830302965
:10BFCF002C203234283030292C2034382830302996
:10BFDF002C3936283030290052562030302020207E
:10BFEF0020202D20526561642076657273696F6E13
:10BFFF0000525520202020202020202D2052656126
:10C00F006420756E69742073697A6500525320201D
:10C01F002020202020202D20526573657420556E1E
:10C02F006974004153206E6E2C6D6D20202D2043BE
:10C03F006F6E6E65637420617564696F20696E70D1
:10C04F007574206E6E20746F206F75747075742008
:10C05F006D6D004141206E6E20202020202D204349
:10C06F006F6E6E65637420617564696F20696E70A1
:10C07F007574206E6E20746F20616C6C206F7574F8
:10C08F007075747300414F206E6E20202020202D7C
:10C09F00205265616420617564696F20636F6E6EF5
:10C0AF00656374696F6E20666F72206F757470753B
:10C0BF0074206E6E00414D206E6E2C6D7520202DFC
:10C0CF0020536574206D75746520737461746520D9
:10C0DF00666F72206F7574707574206E6E002020FD
:10C0EF002020202020202020202020206D75287443
:10C0FF006520537461746529203D202830303D55EB
:10C10F004E4D5554452C2030313D4D555445290049
:10C11F004156206E6E2C767620202D20536574208C
:10C12F00766F6C756D65206C6576656C20666F72C9
:10C13F00206F7574707574206E6E004152206E6E94
:10C14F0020202020202D2052656164206D7574659C
:10C15F002C20766F6C756D6520666F72206F75740D
:10C16F00707574206E6E005373206E6E2C6477742E
:10C17F00202D20536574207363616E206D6F64658D
:10C18F00206477656C6C2074696D6520666F722012
:10C19F006F7574707574206E6E20746F2064777471
:10C1AF00002020202020202020202020202020645C
:10C1BF007774203D203030302E2E2E3235352C2006
:10C1CF0030303020746F2064697361626C65205366
:10C1DF0063616E204D6F6465004773206E6E202083
:10C1EF002020202D20476574207363616E206D6FB2
:10C1FF006465206477656C6C2074696D6520666F6B
:10C20F0072206F7574707574206E6E005361206E9E
:10C21F006E20202020202D2041646420616C6C2032
:10C22F00696E7075747320746F205363616E204C48
:10C23F00697374206F66206F7574707574206E6EDD
:10C24F00005363206E6E20202020202D2052656D1C
:10C25F006F766520616C6C20696E707574732066E3
:10C26F00726F6D205363616E204C697374206F661B
:10C27F00206F7574707574206E6E00532B206E6E68
:10C28F002C6D6D20202D2041646420696E707574B3
:10C29F00206D6D20746F205363616E204C69737431
:10C2AF00206F66206F7574707574206E6E00532D3D
:10C2BF00206E6E2C6D6D20202D2052656D6F766572
:10C2CF0020696E707574206D6D2066726F6D2053CE
:10C2DF0063616E204C697374206F66206F75747084
:10C2EF007574206E6E005378206E6E2020202020F3
:10C2FF002D20446973706C6179205363616E204CFB
:10C30F00697374206F66206F7574707574206E6E0C
:10C31F0000435020202020202020202D2043686122
:10C32F006E67652070617373776F72640043747208
:10C33F006C2D58202020202D2045786974005265DF
:10C34F0073657474696E672E005465726D696E61E2
:10C35F0074696E6720436F6E6E656374696F6E2EBE
:10C36F002E2E00456E746572206F6C6420706173A1
:07C37F0073776F72643A004E
:10D35000902299E0FF04F074D52FF582E43421F592
:10D3600083E0227F0212F75C90229CEFF022902251
:10D3700099E0FF04F0741B2FF582E43422F583E07A
:10D380002290229CE0FF90229AE02416F582E43459
:10D3900022F583EFF0902299E004F022902299E0A8
:10D3A000FF12F75C90229DEFF090229CE0229022E9
:10D3B00099E0FF24D3F582E43421F5832290229969
:10D3C000E024D5F9E43421FA7B0190221112CC96A5
:10D3D00090221112CC769022A802CC969021D5E012
:10D3E000645822902299E0FF12F73190229CEFF0CE
:10D3F00022902299E024D4F582E43421F583E022BE
:10D40000E075F06484E5F075F00A842430FF22FEB4
:10D4100024D0FD90229CE02DF090229BE004F0E0CF
:10D42000640322902299E0FE24D6F582E43421F5AB
:10D4300083E024D075F00AA422E014F0E0C3950B39
:10D440002224D075F064A42DFE902299E024D7F513
:10D4500082E43421F583E024D02E2212CC768F8210
:10D4600075830002C91B90229CE075F00AA4F0901D
:10D470002299E0FF24D52290229AE0FF2416F5821B
:10D48000E43422F583E0FE22F583EEF090229AE068
:10D4900004F02290229E541F4420FBE0FFC3745AE4
:10D4A0009F22FFE0FE248EF8A607748E2EF8E6FF7A
:10D4B00074572EF582E43421F583EF22E075F00AEB
:10D4C00084E5F02430FF22EE24D0FBE0FEA3E0FF51
:10D4D0007C007D0A12C97CEB2FFFEC3E2290221BC0
:10D4E000E0644122FFE0FE243DF582E43421F5832F
:10D4F0002290221BE0645322902299E024D522E05E
:10D5000075F064842430FF2290221BE06452229044
:10D5100022997402F0FF2290221BE0644322ED75F1
:10D52000F00A84E5F075F00AA42EFD0F2214F0A392
:10D53000E014F090229CE0C3950D22E014F0E490FA
:10D540002299F022A3E004F0E0C394042290229AEE
:10D55000E0FFC3950B227B017A22791B9022A8025F
:10D56000CC9690229DE090229C22E490229BF0A3F6
:10D57000F02290229BE0D3940322902299E024038E
:10D58000F0229022A512CC768F8275830022E0FFD4
:10D590007E007B017A2179AF22E4F0A374FFF022B0
:10D5A000EE9390229CF0C394412212CC219022A1B0
:0AD5B00002CC2D24D0FFE434FF224A
:10F73100E4FD12D357FC642C601E902215E0FBEF10
:10F74100C39B40037FFF22EC24D0FED394094003E6
:0AF751007FFF2212D51E80DAAF05FB
:01F75B00228B
:10F75C00E4FD12D375FC642C601E902214E0FBEFC8
:10F76C00C39B40037FFF22EC24D0FED394094003BB
:0AF77C007FFF2212D51E80DAAF05D0
:01F786002260
:10F16900E49022BAF0A3F0AA0774D52A12D35AFE62
:10F17900642C601D902215E0FFEAC39F40037FFFC6
:10F18900229022BA12D4C79022BAF0A3EFF00A80D3
:10F19900D89022BAE060069022BA12D5999022BB83
:02F1A900E0FF85
:01F1AB002241
:10F1AC00E49022A5F0A3F0AA07741B2A12D378FED0
:10F1BC00642C601D902214E0FFEAC39F40037FFF84
:10F1CC00229022A512D4C79022A5F0A3EFF00A80BA
:10F1DC00D89022A5E060069022A512D5999022A67F
:02F1EC00E0FF42
:01F1EE0022FE
:10F6AC00902215E0C394035001229021D7E0B42C92
:10F6BC0002D3227F0212F731EFFD7C00BC0205BDA4
:0CF6CC005502D322EF65086002D322C370
:01F6D800220F
:0AFD16007F3F12FC3D7F0D02FC3D13
:0AFD20007F3F12FD577F0D02FD57D3
:0AFD2A007F2A12FC3D7F0D02FC3D14
:0FFC80007F5812FD577F2A12FD577F0D02FD5747
:10FA1D009022A5EFF0D39463400612D4FF12FC3D63
:10FA2D009022A512D40012FC3D9022A512D4BC0246
:02FA3D00FC3D8E
:10FA3F0090229BEFF0D39463400612D4FF12FD5730
:10FA4F0090229B12D40012FD5790229B12D4BC021D
:02FA5F00FD5751
:10FB010090229BEFF012D50012FD5790229B12D448
:0DFB11000012FD5790229B12D4BC02FD573C
:06F4D3009022A512CC9668
:10F4D90012800E9022A9EFF0E49022A8F09022A9C0
:10F4E900E0FF9022A8E0FEC39F50179022A512CCFE
:10F4F900768E8212D460FF12FC3D9022A8E004F0BF
:02F5090080DBA5
:01F50B0022DD
:06F50C0090229B12CC9638
:10F5120012800E90229FEFF0E490229EF090229FA4
:10F52200E0FF90229EE0FEC39F501790229B12CCD8
:10F53200768E8212D460FF12FD5790229EE004F074
:02F5420080DB6C
:01F5440022A4
:0AFD34007F0D12FC3D7F0A02FC3D2A
:10941C00201D03029CB6C21D201103029549902207
:10942C0014E02419F582E43422F583E4F0902155FC
:10943C00E01460341470030294F524026003029C5F
:10944C00AF12D5567A2179C412FA61EF600E12A3CD
:10945C004F7F3E12FC3DC211E4029511740112A51E
:10946C007C7ABE79310294EFE4902299F0902299A3
:10947C00E0241B12D378FF603AC394304006EFD33C
:10948C0094394018EFC394414006EFD3945A400CE2
:10949C00EFC39461400FEFD3947A5009902299E076
:1094AC00D3940F400912A34F12A50C02951112D39D
:1094BC009580BA7B017A22791B12D3D67A21791B3B
:1094CC0012FA837B017A21791B12800EEFC394056B
:1094DC00500812A35F12A50C802B740212A57C7A83
:1094EC00BE794512A4ED029CAF12D5567A21791B98
:1094FC0012FA61EF601612A35F7F3E12FC3DE490FE
:10950C002155F0C211902214F0C2082212FD347AB7
:10951C00BE795F12A38512FD347F3E12FC3DC21151
:10952C00E4902155F07B017A21791B12D3D67A2154
:10953C0079C412FA8312F0E3D210029CAF90221B72
:10954C00E0FF64686008EF6448600302963220080C
:10955C000302963212FD347ABE797E12A38512FD77
:10956C00347ABE798C12A36F7ABE79BC12A4ED7AD0
:10957C00BE79EE12A37A7ABF791812A5237ABF7935
:10958C005012A37A7ABF798B12A5237ABF79B812BD
:10959C00A38E7ABF79E712A55C7AC0790012A38EEC
:1095AC007AC0791B12A55C300C317AC0793212A3C7
:1095BC00A37AC0796212A3A37AC0799412A3DC7A3D
:1095CC00C079C412A3DC7AC079ED12A4127AC179E5
:1095DC001F12A4127AC1794A12A4347AC179761274
:1095EC00A4347AC179B012A43D7AC179E812A43DB1
:1095FC007AC2791B12A4647AC2795012A4647AC21A
:10960C00798A12A4777AC279BD12A4777AC279F5D5
:10961C0012A4987AC3792012A4987BFF7AC3793C60
:10962C0012F4D3029B3C12D5087004A3E06455706D
:10963C0020200803029CAF12A399AF0D12FA1D7FD4
:10964C002C12FC3DAF0B12FA1D7F0D12FC3D029B40
:10965C003C12D5087004A3E0644F70262008030266
:10966C009CAF12D36312D439400512A4A1801012FE
:10967C00A39990229CE0246CF8E604FF12FA1D02D8
:10968C009B3C12D5087004A3E06453701F200803A0
:10969C00029CAF12A41B7AC3794D12A36F7AC379C3
:1096AC005812F4D312FD34D202029CAF300C31129A
:1096BC00D4DD7004A3E0644F7026200803029CAF35
:1096CC0012D36312D439400512A4A1801012A41B2A
:1096DC0090229CE0245CF8E604FF12FA1D029B3CED
:1096EC0012D5087004A3E06443702B200803029C7D
:1096FC00AF12D50F12D365D3946340030298341282
:10970C00A3AC12A570201403029CAFD203D201D2D9
:10971C000DD20E029CAF12D5177004A3E0644370F7
:10972C0022200803029CAF12D50F12D365D3946389
:10973C00400302983412A3AC90229CE0FF12DFE7A6
:10974C00029CAF12D5087004A3E06456706F200819
:10975C0003029CAF12A446E4902299F07AE6793287
:10976C0012A563502190E63212D5A0400AE0FF9476
:10977C005B5004EF4420F090229CE0FF600312FC4D
:10978C003D12D39580D6E4902299F07AE6794F1267
:10979C00A563502190E64F12D5A0400AE0FF945BE0
:1097AC005004EF4420F090229CE0FF600312FBA5D4
:1097BC0012D39580D6E4FF12FC3D029B3C12D517C8
:1097CC007004A3E06442704030082F12D363BF6072
:1097DC00047F03801F90229CE0B430047F0280142D
:1097EC0090229CE0B418047F01800990229CE0B484
:1097FC000C08E4FF12F84E12EBC312A4252014033C
:10980C00029CAFD20F029CAF12D5177004A3E06478
:10981C0041703D200803029CAF12D50F12D365E0B6
:10982C0014F0E0C3950D400612A4C8029B3C12A490
:10983C0025301402D203E4902299F0902299E0FF93
:10984C00C3950B4003029CAF12A4CF12D39580EBAF
:10985C00200C030298E612D4DD7004A3E06441707E
:10986C007930084912D50F12D365E014F0E0C39596
:10987C000D4003029ADE12A4467F3E12FC3D3014CA
:10988C0002D201E4902299F0902299E0FFC3950B4B
:10989C004003029CAFEF541FFB90229CE09022A946
:1098AC00F0E4FD7FFF12D7F812D39580DB12D517A9
:1098BC007004A3E064506003029CAF200803029C78
:1098CC00AF12FD347BFF7AC3797212F4D312FD34DC
:1098DC00D211E4902155F0029CAF12D5177004A35D
:1098EC00E064537041200803029CAF12D363E490F0
:1098FC002299F012D36EB42CFA12D39C12D52D509F
:10990C0007A3E0C3950B4003029ADE90229DE0FF73
:10991C0012A4CF12A46D7F3E12FC3D201403029CB6
:10992C00AFD203029CAF300C4A12D4DD7004A3E01A
:10993C006453703F200803029CAF12D363E490225F
:10994C0099F012D36EB42CFA12D39C12D52D500769
:10995C00A3E0C3950B4003029ADE12A46D7F3E1266
:10996C00FC3D90229D12A450201403029CAFD20106
:10997C00029CAF300C5812D4DD7004A3E0644D701F
:10998C004D200803029CAF12D363E4902299F0128D
:10999C00D36EB42CFA12D39C12D43A5007A3E0C362
:1099AC0094024003029ADE12A4A87F3E12FC3D12E0
:1099BC00D5626007E0541F44608005E0541F4440AA
:1099CC0012A53F201403029CAFD20D029CAF200CB9
:1099DC0003029A6212D4DD7004A3E06456707720FF
:1099EC000803029CAF12D363E4902299F012D36E59
:1099FC00B42CFA12D39C12D43A5007A3E0C394644B
:109A0C004003029ADE12A4A812D56212D4E4EFF03D
:109A1C00EFC3945A400690229D745AF0301209EE0E
:109A2C0090229D12D496801B90229DE0C3941C50D2
:109A3C0003741CF090229CE0541F4420FBA312D40E
:109A4C009BC31312A4DF7F3E12FC3D201403029C27
:109A5C00AFD20D029CAF300C4C12D4DD7004A3E0DD
:109A6C0064527041200803029CAF12D36312D439A4
:109A7C004003029ADE12A5197F3012FC3D90229C05
:109A8C00E0243CF8E630E7047F3180027F3012FCA2
:109A9C003D7F2C12FC3D90229CE012D4E7E0FF129B
:109AAC00FA1D029CA712D4F17004A3E064737042F7
:109ABC00200803029CAF12D36312D53B12D36EB4B1
:109ACC002CFA902299E0FF12F1AC12D3A4C3950B9F
:109ADC00400612A4C8029CA712A51912D56212D472
:109AEC00A2F07F3E12FC3D201403029CAFD20E026A
:109AFC009CAF90221BE064477004A3E06473703346
:109B0C00200803029CAF12D36312D439400512A56E
:109B1C004C801D12A58690229CE0248EF8E612D56E
:109B2C000012A53312D40112A53312D4BD12FC3D80
:109B3C00029CA712D4F17004A3E06478706D200825
:109B4C0003029CAF12D36312D439400512A54C808A
:109B5C005712A5869022A112CC4500000001E4907A
:109B6C002299F0902299E0C3950D503C90229CE0F4
:109B7C0025E025E02468F582E43421F58312D5AA8A
:109B8C0012CBB6EC4D4E4F60047F7880027F6F1283
:109B9C00FC3D9022A112CC21780112CC0E9022A176
:109BAC0012CC3912D39580BB029CA712D4F170044D
:109BBC00A3E064617020200803029CAF12D36312EF
:109BCC00D439400512A590800A12A48012CC45FF0E
:109BDC00FFFFFF029CA712D4F17004A3E064637032
:109BEC0020200803029CAF12D36312D43940051213
:109BFC00A590800A12A48012CC4500000000029CA3
:109C0C00A712D4F17004A3E0642B703B200803026C
:109C1C009CAF12D36312D53B12D36EB42CFA12A4A0
:109C2C00B2950B5006A3E0950D400512A4F48014D8
:109C3C0012A3E5C083C08212D5AA12CBC3D082D0A6
:109C4C008312CC39029CA712D4F17004A3E0642DCA
:109C5C00704030084E12D36312D53B12D36EB42C25
:109C6C00FA12A4B2950B5006A3E0950D400512A470
:109C7C00F4801D12A3E5C083C08212CC2D9022A1CA
:109C8C0012CC2112CBDD12CBB6D082D08312CC39C0
:109C9C00800930080E12FD3412FD1612FD347F3E81
:109CAC0012FC3DE4902214F0C20820060302A34EDD
:109CBC00C20612D3DC7004A3E06453703620083360
:109CCC0012F6AC500302A349E4902299F012D3503F
:109CDC00B42CFA12D3E3C39400500302A349E0D38B
:109CEC009403400302A34912A52A12F84E12EBC3A7
:109CFC0002A34912D3DC7004A3E0644C7035200835
:109D0C003212F6AC500302A349E4902299F012D31C
:109D1C0050B42CFA12D3E3D3940F5006E0C3940141
:109D2C00500612FD2002A34912A52AF50812F89636
:109D3C0002A34912D3DC7004A3E064416003029DCA
:109D4C00F2300803029DF212F6AC500302A349E470
:109D5C00902299F012D350B42CFAE490229AF0127B
:109D6C00D56A12D4F812D35AFF642E6051EF642CCA
:109D7C00604C12D46612D35A12D40F703174D32F94
:109D8C0012D3B5E0FFD394325029EFB4320812D37A
:109D9C00F1D39435501D12D3AEE0B4321174D42FDC
:109DAC0012D3F7B43508EED394354002800512D5A2
:109DBC0072400512FD20800612D395029D6E12D3BF
:109DCC008112D5444099E490229AF012D47774AB66
:109DDC002FF582E4342112D488E0B404EE12FC8016
:109DEC0012F3EB02A34912D3DC7004A3E0644D60C0
:109DFC0003029EA5300803029EA512F6AC50030286
:109E0C00A349E4902299F012D350B42CFAE4902296
:109E1C009AF012D56A12D4F812D35AFF642E6051FC
:109E2C00EF642C604C12D46612D35A12D40F7031DA
:109E3C0074D32F12D3B5E0FFD394325029EFB43240
:109E4C000812D3F1D39435501D12D3AEE0B43211B5
:109E5C0074D42F12D3F7B43508EED3943540028066
:109E6C000512D572400512FD20800612D395029E74
:109E7C002112D38112D5444099E490229AF012D445
:109E8C007774512FF582E4342112D488E0B404EEB7
:109E9C0012FC8012F45F02A34912D3DC7004A3E01D
:109EAC0064476003029F58300803029F5812F6ACB7
:109EBC00500302A349E4902299F012D350B42CFA27
:109ECC00E490229AF012D56A12D4F812D35AFF6495
:109EDC002E6051EF642C604C12D46612D35A12D4FB
:109EEC000F703174D32F12D3B5E0FFD394325029B5
:109EFC00EFB4320812D3F1D39435501D12D3AEE027
:109F0C00B4321174D42F12D3F7B43508EED3943580
:109F1C004002800512D572400512FD20800612D336
:109F2C0095029ED412D38112D5444099E490229A82
:109F3C00F012D47774C02FF582E4342112D488E067
:109F4C00B404EE12FC8012F49902A34912D3DC7013
:109F5C0004A3E06450703320083012F6AC500302B6
:109F6C00A349902215E012D3B3E4F0902299F01299
:109F7C00D350B42CFA12D3BD7B017A2179C412FAD6
:109F8C008312FC8012F0E302A34912D3DC7004A309
:109F9C00E06443705320085012F6AC500302A349FE
:109FAC00E4902299F012D350B42CFA12A50312D5D6
:109FBC004D400302A34912D423FD74D52E12D35A5B
:109FCC0012D441FE90229CF0746C2FF8E66E600F58
:109FDC0090229CE0FDE49022A9F07BFF12D7F812AE
:109FEC00D57AA3E004F080C612D3DC7004A3E0643D
:109FFC0056702720082412F6AC500302A349E490B3
:10A00C002299F012D350B42CFA12D3E312FC8090A4
:10A01C00229CE0FF12DFE702A34912D3DC7004A3F9
:10A02C00E06452702E20082B12F6AC500302A349A8
:10A03C00E4902299F012D350B42CFA12D3E312FC10
:10A04C008012A57020140302A349D203D201D20EB0
:10A05C0002A34912D3DC7004A3E0645470332008CB
:10A06C003012F6AC500302A349902215E012D3B380
:10A07C00E4F0902299F012D350B42CFA12D3BD7B99
:10A08C00017A21792C12FA8312FC8012F12602A398
:10A09C004912D3DC7004A3E06459600302A131308F
:10A0AC00080302A13112F6AC500302A349E490223A
:10A0BC0099F012D350B42CFA12D39512D3E612D3D2
:10A0CC0050B42CFA12D4F8F9E43421FA7B01902222
:10A0DC001112CC9612D350B42CFA12D4F812D35AC3
:10A0EC0090229CB4310812D58E12EA83800612D5C8
:10A0FC008E12E79212FC8012F425902299E014F053
:10A10C00E024D5F582E43421F583E4F012D3D07B3E
:10A11C00017A2179B312FA8390229CE0FF7E00121F
:10A12C00EC7E02A349300C5512D3DC7004A3E0641E
:10A13C0061704A20084712F6AC500302A349E49020
:10A14C002299F012D350B42CFA12A50312D54D401B
:10A15C000302A34912D423FD74D52E12D35A12D460
:10A16C0041FE90229CF0745C2FF8E66E6006902203
:10A17C009A12A45012D57AA3E004F080CF200C03DD
:10A18C0002A24212D3DC7004A3E06476600302A244
:10A19C004230080302A24212F6AC500302A349E477
:10A1AC00902299F012D350B42CFA12A55312D54D1B
:10A1BC00400302A34912D4F812D35AB4300F743CA2
:10A1CC002FF8747F56F6EF541F4440801190229A5A
:10A1DC00E0FF243CF8748046F6EF541F446012A54F
:10A1EC003F902299E0FF12D428FE74D72F12D44F3F
:10A1FC0090229EF0E090229A12D4E4EFF0EFC394F8
:10A20C005A400690229E745AF0301206EE12D493E5
:10A21C00801590229EE0C3941C5003741CF0902275
:10A22C009AE012D493C31312A4DF12D57A12F6D982
:10A23C0012D48C02A1B912D3DC7004A3E064737045
:10A24C007A20087712F6AC500302A349E4902299C5
:10A25C00F012D350B42CFA12A55390229AE0C39565
:10A26C000B400302A34912D35012D5B3FE7C007DE0
:10A27C006412C97C90229FEEF0A3EFF012D350121F
:10A28C00D5B3FE7D0A12C97C90229FEE8FF012C9C5
:10A29C00C412D35012D5B390229F8FF012C9C49020
:10A2AC00229FE0600690229F12D5999022A0E09008
:10A2BC00229A12D4A212D48B02A2669021D5E0B4B9
:10A2CC005818A3E0B442132008109027FF7401F033
:10A2DC00C2AF53D0FD121000806312D3DC7004A304
:10A2EC00E06445705020084D12F6AC4050E49022CA
:10A2FC0099F012D350B42CFA12FC80E490229AF00C
:10A30C0090229AE0FDC3950B5033902299E0FE0405
:10A31C00F074D52E12D35A24D090229CF0E0700306
:10A32C00FF80027F0174882DF582E43422F583EFDF
:10A33C0012D48B80CB12F6AC400312FD16E49022A3
:02A34C0015F00A
:10A34E002212FD347BFF7ABE791F12F4D312FD3434
:10A35E002212FD347BFF7ABE791F12F4D312FD3424
:10A36E00227BFF12F4D312FD347BFF227BFF12F40B
:10A37E00D312FD347BFF227BFF12F4D312FD342265
:10A38E007BFF12F4D312FD347BFF2212FD3412FD3B
:10A39E002A12FD34227BFF12F4D312FD342212FD59
:10A3AE003412FD2A12FD3490229CE075F00A8424AA
:10A3BE0030FF12FC3D90229CE075F00A84E5F024FB
:10A3CE0030FF12FC3D12FD347F3E12FC3D227BFF1E
:10A3DE0012F4D312FD342212FD3412FD2AE47F0151
:10A3EE00FEFDFC90229DE0F9F812CC0E9022A112F7
:10A3FE00CC3990229CE025E025E02468F582E434F7
:10A40E0021F583227BFF12F4D312FD342212FD3488
:10A41E0012FD2A12FD342212FD3412FD2A12FD34D1
:10A42E007F3E12FC3D227BFF12F4D312FD34227BC1
:10A43E00FF12F4D312FD342212FD3412FD2A12FD46
:10A44E003422E0541FFB90229CE09022A9F0E4FD00
:10A45E007FFF12D7F8227BFF12F4D312FD342212A3
:10A46E00FD3412FD2A12FD34227BFF12F4D312FDAD
:10A47E00342212FD3412FD2A90229CE025E025E0C4
:10A48E002468F582E43421F583227BFF12F4D31283
:10A49E00FD342212FD3412FD162212FD3412FD2A55
:10A4AE0012FD3422902299E0FF12F1AC90229DEF22
:10A4BE00F0E014F090229CE0C32212FD3412FD163F
:10A4CE002290229CE0FDE49022A9F07BFF12D7F8A7
:10A4DE0022547F9022A9F0E4FD7FFF12D7F82212BA
:10A4EE00F4D312FD342212FD3412FD1612FD347F08
:10A4FE003E12FC3D2212FC80E490229AF0227F3E16
:10A50E0012FC3DE4902155F0C2112212FD3412FDD1
:10A51E002A12FD342212F4D312FD342212FC809042
:10A52E00229CE0FF2212FC3D90229CE0248EF8E655
:10A53E0022FBE49022A9F0FD7FFF12D7F82212FD34
:10A54E003412FD162212FC80E490229AF02212F4AC
:10A55E00D312FD34227BFF12800E902299E0FEC3AF
:10A56E009F2290229CE0FF12D0B612E6722290211A
:10A57E0055F012FD347BFF2212FD3412FD2A12FD1E
:09A58E00342212FD3412FD1622E4
:06FA61009022A512CC96D4
:10FA6700E4FF9022A812D45BFE9022A512D45BB5C6
:0BFA770006077002FF220F80E97F01EC
:01FA82002261
:06FA83009022A512CC96B2
:10FA8900E4FF9022A812D45BFE600A12D582EE121E
:0CFA9900C95A0F80ED12D582E402C95A50
:06800E009022AA12CC969C
:0D801400E4FF9022AA12D45B60030F80F5F8
:01802100223C
:10F01300902257E0FF04F0745E2FF582E43422F56A
:10F023008322902215E0FF04F074D52FF582E43497
:10F0330021F583742CF022902214E0FF04F0741B5A
:10F043002FF582E43422F583742CF0227E007F3C7A
:07F053007D007B0102CCE50A
:10FC1800C2CAC2AD43874CE4F5C875CA7E75CBFF2E
:03FC2800D2CA221B
:10F1EF0012FC18C2DFD2DEC2DDC2D9C2D875920CB2
:10F1FF0075930CD2C3D2C2AFD9902299E4F0A3EF8A
:10F20F00F0D2DC43A710C209C2067A2179D512F0D9
:10F21F004F7A22791B12F04FE4902215F0902214AE
:01F22F00F0EE
:01F2300022BB
:03804B0002E10F40
:10E10F00C0E0C083C082C0D075D000C006C0072059
:10E11F00D80302E1F590214FE5D9F0E0FFB4810576
:10E12F00D20B02E1F3EFB4D905D20402E1F3EF64AD
:10E13F008A700302E1F3EF30E71464816010EF643B
:10E14F00D9600BD208EF547F90214FF08002C208A4
:10E15F0090214FE0FF641B6006EF6003B4FF1420B3
:10E16F000807902215E4F08005902214E4F0C2080D
:10E17F0002E1F3EF640D701820080B12F02512F076
:10E18F0025D20602E1F312F03A12F03AD21D805472
:10E19F0090214FE0FFB42004C208804820081C9053
:10E1AF002215E0C3943A500EE0FE04F074D52EF51C
:10E1BF0082E4342180229022158026902214E0C31D
:10E1CF00943A501A90214FE0FF902214E0FE04F091
:10E1DF00741B2EF582E43422F583EFF08006902233
:10E1EF0014743AF0C2D830D904C209C2D9D007D0BA
:0AE1FF0006D0D0D082D083D0E032E9
:10FC3D002009FD300807EF4480F5D980028FD9D215
:02FC4D0009228A
:08FD57002009FDD2098FD92219
:10F3320012EBC3C29FD29EC29DC299C2987591031D
:10F34200D2B1D2B0AF99902299E4F0A3EFF0D29C5F
:10F35200D2ACC207C205C218C2197E007F207D004E
:0EF362007B017A22795E12CCE5E4902257F00E
:01F37000227A
:0380230002E992DD
:10E99200C0E0C083C082C0D075D000C006C00730BE
:10E9A200985590214DE599F0C298E0FF641B6006EE
:10E9B200EF6003B4FF07902257E4F0803AEFB40D02
:10E9C2001012F013742CF012F013742CF0D2058094
:10E9D2002690214DE0FF6420601D902257E0C394F1
:10E9E2001E500EE0FE04F0745E2E12F01DEFF08059
:10E9F20006902257741EF0309904C207C299D007BC
:0BEA0200D006D0D0D082D083D0E0320C
:10FBA5002007FDD2078F99EF640D600CEFC39430E9
:09FBB5004006EFD3943950002200
:10F2B3009022A612CC39C28EC2AB43878053890FEA
:10F2C3004389209022AAE0FEA3E0FFE4FCFD7BC07B
:10F2D300FAF9F812CA99A804A905AA06AB0790225D
:10F2E300A612CC2112CB24EFF40414F58DD28E2276
:10FB1E0090229AE02457F582E43421F5832212CC08
:0DFB2E000E90229E02CC3990229E02CC2126
:10DA0700782BE6D39400500302DB92E4F690229938
:10DA1700F0A3F0C390229AE0950B7480F8902299B6
:10DA2700E0648098400302DB92A3E0FF248EF8E6CF
:10DA3700700302DB7F74882FF582E43422F583E0DC
:10DA47006401600302DB7F12FB1EE014F074572FA2
:10DA570012FB24E0600302DB8590229AE0FFE6FEDA
:10DA670074572F12FB24EEF090229AE0246CF8E60C
:10DA77002401FFE433AB07FAC3EB950D7480F86A12
:10DA8700984003E4FAFBE47F01FEFDFCA903A8012B
:10DA970012FB2C90229BE4F0A304F0902299E0FE65
:10DAA700A3E07802C333CE33CED8F92468F5827465
:10DAB700213EF58312CC2190229E12CC2D12CBB69B
:10DAC700E4FBFAF9F8C312CBEA706BC390229CE02F
:10DAD700950D7480F890229BE0648098505812FB53
:10DAE70035780112FB2CE50DB4040912FB35EF5410
:10DAF7000FFF8008E50DB4080712FB35E4FE800927
:10DB0700E50DB4100912FB35E4FDFC12FB2FE4FF11
:10DB1700FEFDFC90229E12CC2DC312CBEA700A9018
:10DB2700229E12CC450000000190229BE475F00173
:10DB370012C9C402DAA290229AE0246CF890229CBF
:10DB4700E026A3F0C3950D4004E0950DF090229ACE
:10DB5700E0FF90229DE0FD300C0BEF541FFB90225D
:10DB6700A9EDF08007E49022A9F07BFF12D7F830E7
:10DB7700140CD203D201800612FB1E7401F090220E
:0BDB870099E475F00112C9C402DA1A1B
:01DB92002270
:0380000002E7068E
:0CE70600787FE4F6D8FD75819D02E74D98
:05800600782AA6092202
:10F61E00782AE665096029A609788DE618466007FE
:10F62E0008E61618700116782808E6161886067071
:10F63E0001164E700B782B7601782876070876D057
:01F64E002299
:0BFCD90074B62FF582E43422F583227C
:07FD660012FCD9E50AF022AE
:10F7870012FCD9E0FF2DFED39F400FE50A9F4006EC
:10F79700E50AD39E4002D322C322E50AC39F50093C
:0AF7A700E50AC39E4003D38001C3AE
:01F7B1002235
:03800B0002FC4F25
:10FC4F00C28C758CF3758A0CC28DD28C1509050A7E
:01FC5F003272
:10FC0200C28DAF89EF54F04401F589758A0C758C69
:05FC1200F3D2A9D28C21
:01FC170022CA
:0CFCB70052766F0052766100534D2D0014
:06F7FC004122BC00C11E09
:10EEAF009021ABE075F06484E5F075F00A842430AE
:10EEBF00FF229021ABE075F00A84E5F02430FF22A9
:10EECF009021ABE075F064842430FF22E490213C64
:10EEDF00F0C20422E0243DF582E43421F583E0FF03
:08EEEF002290211AE004F02238
:10B49A00902167E012CCBFB52300B53701B554023D
:10B4AA00B57D03B59A04B5BC05B5E406B60607B67C
:10B4BA008108B6A309B7210AB7430BB7C50CB7E78A
:10B4CA000DB8060EB8280FB84A10B86C11B8841215
:10B4DA00B8A613B8D614B8F815B91716B93D17B9DE
:10B4EA008F18B9C819B9F71ABA191BBA441CBA7015
:10B4FA001DBAA61EBAC91FBB0F20BB3221BB6C22C4
:10B50A00BB8F23BBD924BBFC25BC4826BC7327BCF4
:10B51A008D28BCA7290000BCB2200B0302BCB77F50
:10B52A005812FD577F2A12BCD77401F0227F581295
:10B53A00FD577F4512BCD77402F0D214E4FF12FD06
:10B54A0066301E0302BCB702BC402004079022BC2E
:10B55A00E0B40A0F9021677403F0C204C20BD2143C
:10B56A00C21E2212BCF7400302BCB79021677401C5
:10B57A0002BC6B7F5812FD577F4C12FD57AF081261
:10B58A00BDDD740412BCE3301E0302BCB702BC402A
:10B59A002004079022BCE0B40A08902167740502CF
:10B5AA00BAB512BCF7400302BCB790216774030214
:10B5BA00BC6B12F872902299EFF07F5812FD577FF8
:10B5CA005312FD57902299E0FF12BDDD740612BC9A
:10B5DA00E3301E0302BCB702BC402004079022BC21
:10B5EA00E0B40A08902167740702BAB512BCFF409A
:10B5FA000302BCB7902167740502BC6B7F5812FD29
:10B60A00577F4112FD5712EECF12FD5712EEAF12BD
:10B61A00FD5712EEC112BD3D9021AC12EED212FDC1
:10B62A00579021AC12EEB212FD579021AC12EEC423
:10B63A0012BD3D9021AD12EED212FD579021AD12EE
:10B64A00EEB212FD579021AD12EEC412BD4E9021FA
:10B65A00AE12EED212FD579021AE12EEB212FD5783
:10B66A009021AE12EEC412BDB0740812BCED301EA9
:10B67A000302BCB702BC402004079022BCE0B40A13
:10B68A0008902167740902BAB512BCFF400302BCD4
:10B69A00B7902167740702BC6B7F5812FD577F4D24
:10B6AA0012BE0A12EED212BE0A12EEB212FD579062
:10B6BA00215112EEC412BD4E90215212EED212FD49
:10B6CA005790215212EEB212FD5790215212EEC437
:10B6DA0012BD7690215312EED212FD5790215312C9
:10B6EA00EEB212FD5790215312EEC412BD7690218C
:10B6FA005412EED212FD5790215412EEB212FD5797
:10B70A0090215412EEC412BDB0740A12BCED301E60
:10B71A000302BCB702BC402004079022BCE0B40A72
:10B72A0008902167740B02BAB512BD11400302BC1E
:10B73A00B7902167740902BC6B7F5812FD577F4787
:10B74A0012BE1112EED212BE1112EEB212FD5790B3
:10B75A0021C012EEC412BDE69021C112EED212FD32
:10B76A00579021C112EEB212FD579021C112EEC4B8
:10B77A0012BDE69021C212EED212FD579021C212DA
:10B78A00EEB212FD579021C212EEC412FD577F2E5F
:10B79A0012BE1812EED212BE1812EEB212FD579055
:10B7AA0021C312EEC412FD577F0D12FD57740C12FD
:10B7BA00BD07301E0302BCB702BC4020040790221A
:10B7CA00BCE0B40A08902167740D02BAB512BD1123
:10B7DA00400302BCB7902167740B02BC6B7F5812FE
:10B7EA00FD577F5012BD7F7A2179C412BDFF740EB6
:10B7FA0012BD07301E0302BCB702BC4020040790EA
:10B80A0022BCE0B40A08902167740F02BAB512BDCF
:10B81A0023400302BCB7902167740D02BC6B7F58AA
:10B82A0012FD577F4912FD57AF0D12FA3F7F0D12D5
:10B83A00FD57741012BD19301E0302BCB702BC407A
:10B84A002004079022BCE0B40A0890216774110210
:10B85A00BAB512BD23400302BCB7902167740F0228
:10B86A00BC6B7F5812FD577F4F12BCC6741212BDB3
:10B87A00F8301E0302BCB702BC402004079022BC69
:10B88A00E0B40A08902167741302BAB512BD2B40BE
:10B89A000302BCB7902167741102BC6B7F5812FD7A
:10B8AA00577F4312BD7F90211AE0C3950B500A12AD
:10B8BA00BDA6246C12BD6980ED7F0D12FD5774146C
:10B8CA0012BD19301E0302BCB702BC402004079007
:10B8DA0022BCE0B40A08902167741502BAB512BDF9
:10B8EA002B400302BCB7902167741302BC6B7F58CC
:10B8FA0012FD577F5412FD577A21792C12BDFF741D
:10B90A001612BD33301E0302BCB702BC4020040726
:10B91A009022BCE0B40A0CC204E490211A12BDCEF3
:10B92A00C21E2212BD46400302BCB790216774159D
:10B93A0002BC6B7F5812FD577F5912FD5712BDA6E4
:10B94A00FF12FA3F7F2C12FD577B017A2179B3123D
:10B95A00F50C7F2C12FD5790211AE0FF7E007B0127
:10B96A007A2179AF12E49550047F3180027F301238
:10B97A00FD577F0D12FD57741812BD33301E030296
:10B98A00BCB702BC402004089022BCE0640A701EC6
:10B99A00C204E50D14FF90211AE0C39F5007E0048A
:10B9AA0012BDCE80069021677419F0C21E2212BD04
:10B9BA0046400302BCB7902167741702BC6B7F58DC
:10B9CA0012FD577F4612FD577BFF200C067AFC7941
:10B9DA00B780047AFC79BB12F50C7F0D12FD5774FF
:10B9EA001A12BD57301E0302BCB702BC402004071E
:10B9FA009022BCE0B40A08902167741B02BAB512FF
:10BA0A00BD61400302BCB7902167741902BC6B7F09
:10BA1A005812FD577F4812FD577BFF7AFC79BF12F7
:10BA2A00F50CAF0D12FA3F7F5812BCC6741C12BD3A
:10BA3A00F8301E0302BCB702BC402004079022BCA7
:10BA4A00E0B40A12902167200C067421F002BC5857
:10BA5A00741DF002BC5812BD61400302BCB79021AC
:10BA6A0067741B02BC6B7F5812FD577F6112BDEFD2
:10BA7A0090211AE0C3950B50107F3012FD57902188
:10BA8A001AE0245C12BD6980E77F0D12FD57741E0F
:10BA9A0012BD57301E0302BCB702BC4020040790F7
:10BAAA0022BCE0B40A09902167741FF002BC581244
:10BABA00BD88400302BCB7902167741D02BC6B7F2E
:10BACA005812FD577F7612BDEF90211AE0FFC395F9
:10BADA000B501F743C2FF8E630E7047F3180027F59
:10BAEA003012FD5790211A12EEE312FA3F12EEF0CD
:10BAFA0080D77F0D12FD57742012BD9C301E0302A1
:10BB0A00BCB702BC402004079022BCE0B40A0990EA
:10BB1A0021677421F002BC5812BD88400302BCB7E9
:10BB2A00902167741F02BC6B7F5812FD577F7312F6
:10BB3A00FD57E490211AF090211AE0FFC3950B50AB
:10BB4A000E748E2FF8E6FF12FB0112EEF080E87FEA
:10BB5A000D12FD57742212BD9C301E0302BCB7029F
:10BB6A00BC402004079022BCE0B40A099021677403
:10BB7A0023F002BC5812BDB9400302BCB79021673A
:10BB8A00742102BC6B7F5812FD577F6612BD9074F8
:10BB9A0001F07AE6794F12BDC1FEC39F501DEE90A7
:10BBAA00E64F93B420047F1F800990211AE090E6A3
:10BBBA004F93FF12FD5712EEF080D712BCB87424CF
:10BBCA00F0E4FF12FD66301E0302BCB702BC40203F
:10BBDA0004079022BCE0B40A099021677425F00298
:10BBEA00BC5812BDB9400302BCB790216774230246
:10BBFA00BC6B7F5812FD577F6412BD907401F07AB6
:10BC0A00E6793212BDC1FEC39F501DEE90E6329313
:10BC1A00B420047F1F800990211AE090E63293FF36
:10BC2A0012FD5712EEF080D712BCB87426F0E4FF6A
:10BC3A0012FD66201E77E49022BCF0D21E22200458
:10BC4A00079022BCE0B40A0B9021677427F0C20463
:10BC5A00C21E227DC8E4FF12F787505190216774F3
:10BC6A0025F09022BCE004F0227F5812FD577F583D
:10BC7A0012FD577F0D12FD579021677428F0E4FFDB
:10BC8A0002FD66300407902167742980177DC8E495
:10BC9A00FF12F78750179021677427F022300B0D97
:0DBCAA00E4902167F0C20422E4902167F0CD
:10BCB70022E4FF12FD577F0D12FD579021672212D4
:10BCC700FD57AF0B12FA3F7F0D12FD5790216722E8
:10BCD70012FD577F0D12FD5790216722902167F0C3
:10BCE700E4FF12FD6622902167F0E4FF12FD662251
:10BCF7007DC8E4FF12F787227DC8E4FF12F7872289
:10BD0700902167F0E4FF12FD66227DC8E4FF12F779
:10BD17008722902167F0E4FF12FD66227DC8E4FFC9
:10BD270012F787227DC8E4FF12F78722902167F078
:10BD3700E4FF12FD662212FD577F2E12FD57227D6A
:10BD4700C8E4FF12F7872212FD577F2E12FD5722F4
:10BD5700902167F0E4FF12FD66227DC8E4FF12F729
:10BD67008722F8E6FF12FA3F90211AE004F0221228
:10BD7700FD577F2E12FD572212FD57E490211AF02E
:10BD8700227DC8E4FF12F7872212FD577F1F12FD9D
:10BD97005790211A22902167F0E4FF12FD66227F57
:10BDA7003012FD5790211AE02212FD577F0D12FD28
:10BDB70057227DC8E4FF12F787227BFF12800EEF20
:10BDC70014FF90211AE022F0E0FF7E0012EB609052
:10BDD70021677417F02212FA3F7F0D12FD572212C6
:10BDE700FD577F2E12FD572212FD57E490211AF0BE
:10BDF70022F0E4FF12FD66227B0112F50C7F0D1283
:10BE0700FD572212FD579021512212FD579021C054
:08BE17002212FD579021C32205
:10C38600300A3F902156E014601B04702F12C8201B
:10C396007F4C12FD57AF0812FA3F7F0D12FD5790E2
:10C3A600215602C7F930040AE4902156F0C204C2AD
:10C3B6000A2212C828400302C81F8000E4902156B2
:10C3C600F022300F4A9021A9E014602604703A1238
:10C3D600F872902299EFF012C8207F5312FD579001
:10C3E6002299E0FF12FA3F7F0D12FD579021A90214
:10C3F600C7F930040AE49021A9F0C204C20F221240
:10C40600C828400302C81F8000E49021A9F022300A
:10C41600034D902150E014602904703D12C8397F05
:10C426004312C89490229AE0C3950B500A12C8C1D1
:10C43600246C12C88780ED7F0D12FD5790215002A3
:10C44600C7F930040AE4902150F0C204C203221254
:10C45600C841400302C81F8000E4902150F02230FA
:10C466000C4E30014B90214EE014602904703E12B0
:10C47600C8397F6112C89490229AE0C3950B500A7E
:10C4860012C8C1245C12C88780ED7F0D12FD57903B
:10C49600214E02C7F930040AE490214EF0C204C2CC
:10C4A600012212C841400302C81F02C52102C5214C
:10C4B600300C6E300D6B90214EE014604704705BBB
:10C4C60012C8527F7612FD57E490229AF090229A73
:10C4D600E0FFC3950B5022743C2FF8E630E7047F4B
:10C4E6003180027F3012FD5790229A12EEE312FA43
:10C4F6003F90229AE004F080D47F0D12FD579021E0
:10C506004E02C7F930040AE490214EF0C204C20D6F
:10C516002212C85A400302C81F8000E490214EF040
:10C526002230103A9021AAE014601804702D12C827
:10C53600527F5012FD577A2179C412C8B69021AAAB
:10C5460002C7F930040AE49021AAF0C204C21022FC
:10C5560012C85A400302C81F02C7D202C7D220150A
:10C566000302C5FC90213CE014607404600302C51C
:10C57600F912C86E7F4112FD5712EECF12FD571207
:10C58600EEAF12FD5712EEC112C8309021AC12EE7A
:10C59600D212FD579021AC12EEB212FD579021AC8B
:10C5A60012EEC412C8309021AD12EED212FD579091
:10C5B60021AD12EEB212FD579021AD12EEC412C893
:10C5C600499021AE12EED212FD579021AE12EEB274
:10C5D60012FD579021AE12EEC412C86202C7F9309E
:10C5E600040612EEDBC2152212C876400302C81FEB
:10C5F60002C76F02C76F20170302C69790213CE05F
:10C6060014607704600302C69412C86E7F4D12C888
:10C61600CB12EED212C8CB12EEB212FD57902151B8
:10C6260012EEC412C84990215212EED212FD579052
:10C63600215212EEB212FD5790215212EEC412C8C8
:10C646007E90215312EED212FD5790215312EEB274
:10C6560012FD5790215312EEC412C87E9021541237
:10C66600EED212FD5790215412EEB212FD579021D0
:10C676005412EEC412C86202C7F930040612EEDB89
:10C68600C2172212C876400302C81F02C76F02C72C
:10C696006F20160302C73A90213CE014700302C7CC
:10C6A6002504600302C73812C89D7F4712C8D212FC
:10C6B600EED212C8D212EEB212FD579021C012EE7F
:10C6C600C412C8AD9021C112EED212FD579021C1FD
:10C6D60012EEB212FD579021C112EEC412C8AD90EF
:10C6E60021C212EED212FD579021C212EEB212FDF5
:10C6F600579021C212EEC412FD577F2E12C8D912CE
:10C70600EED212C8D912EEB212FD579021C312EE24
:10C71600C412FD577F0D12FD5790213C02C7F93018
:10C72600040612EEDBC2162212C8A5400302C81F79
:10C736008037803530003890213CE0146018047052
:10C746002812C89D7F5412FD577A21792C12C8B63B
:10C7560090213C02C7F930040612EEDBC200221219
:10C76600C8A5400302C81F8000E490213CF0223097
:10C776000E609021AAE014603B047050C2047F58FA
:10C7860012FD577F7312FD57E490229AF090229A79
:10C79600E0FFC3950B5011748E2FF8E6FF12FB01D4
:10C7A60090229AE004F080E57F0D12FD579021AAB1
:10C7B6007401F02230040AE49021AAF0C204C20EE9
:10C7C600227DC87F0112F787504F8000E49021AA8E
:10C7D600F0223002449021A8E014601E047035C295
:10C7E600047F5812FD577F5A12FD577F0D12FD57D1
:10C7F6009021A87401F0FF02FD6630040CE490213C
:10C80600A8F0C202C2040200007DC87F0112F787A9
:09C8160050078000E49021A8F015
:10C81F0022C2047F5812FD57227DC87F0112F7876D
:10C82F002212FD577F2E12FD5722C2047F5812FD90
:10C83F0057227DC87F0112F7872212FD577F2E12D4
:10C84F00FD5722C2047F5812FD57227DC87F011267
:10C85F00F7872212FD577F0D12FD5790213C22C200
:10C86F00047F5812FD57227DC87F0112F7872212CD
:10C87F00FD577F2E12FD5722F8E6FF12FA3F902246
:10C88F009AE004F02212FD57E490229AF022C2049B
:10C89F007F5812FD57227DC87F0112F7872212FDA4
:10C8AF00577F2E12FD57227B0112F50C7F0D12FDC3
:10C8BF0057227F3012FD5790229AE02212FD579097
:10C8CF0021512212FD579021C02212FD579021C3F2
:01C8DF002236
:10E7120002E817E493A3F8E493A34003F68001F21E
:10E7220008DFF48029E493A3F85407240CC8C33308
:10E73200C4540F4420C8834004F456800146F6DFD7
:10E74200E4800B010204081020408090F7DCE47E94
:10E75200019360BCA3FF543F30E509541FFEE493CC
:10E76200A360010ECF54C025E060A840B8E493A393
:10E77200FAE493A3F8E493A3C8C582C8CAC583CABE
:10E78200F0A3C8C582C8CAC583CADFE9DEE780BE76
:01F802000005
:10C8E000C2D530F707B2D563F0FF05F030E70CB2E0
:10C8F000D5F4048463F0FF05F080018430D502F4A0
:02C9000004220F
:10C90200BB010689828A83E0225002E722BBFE0233
:09C91200E32289828A83E4932266
:10C91B00BB010CE58229F582E5833AF583E02250D1
:10C92B0006E92582F8E622BBFE06E92582F8E2221B
:0DC93B00E58229F582E5833AF583E4932235
:10C94800BB010689828A83F0225002F722BBFE01CE
:02C95800F322C8
:10C95A00F8BB010DE58229F582E5833AF583E8F013
:10C96A00225006E92582C8F622BBFE05E92582C8BF
:02C97A00F222A7
:10C97C00EF8DF0A4A8F0CF8CF0A428CE8DF0A42ECF
:02C98C00FE2289
:10C98E00C2D5EC30E709B2D5E4C39DFDE49CFCEEC4
:10C99E0030E715B2D5E4C39FFFE49EFE12CD11C35E
:10C9AE00E49DFDE49CFC800312CD1130D507C3E459
:06C9BE009FFFE49EFE2233
:10C9C400C5F0F8A3E028F0C5F0F8E58215827002FE
:06C9D4001583E038F0229B
:10C9DA00BB0110E58229F582E5833AF583E0F5F09B
:10C9EA00A3E0225009E92582F886F008E622BBFE78
:10C9FA000AE92582F8E2F5F008E222E5832AF583BE
:08CA0A00E993F5F0A3E9932282
:10CA1200BB010DC58229C582C5833AC58302C9C43B
:10CA22005011C58229F808E5F026F618F5F0E582DE
:10CA320036F622BBFE11C58229F808E225F0F5F090
:10CA4200F218E23582F222F8E58229F582E5832A9C
:0DCA5200F58374019325F0F5F0E49338228C
:10CA5F00F8BB0111E58229F582E5833AF583E8F009
:10CA6F00E5F0A3F0225009E92582C8F608A6F022C6
:0DCA7F00BBFE09E92582C8F2E5F008F222AD
:0DCA8C00EF2BFFEE3AFEED39FDEC38FC22F9
:10CA9900E88FF0A4CC8BF0A42CFCE98EF0A42CFC3C
:10CAA9008AF0EDA42CFCEA8EF0A4CDA8F08BF0A4BA
:10CAB9002DCC3825F0FDE98FF0A42CCD35F0FCEB19
:10CAC9008EF0A4FEA9F0EB8FF0A4CFC5F02ECD39DE
:0FCAD900FEE43CFCEAA42DCE35F0FDE43CFC224B
:10CAE80075F008758200EF2FFFEE33FECD33CDCC05
:10CAF80033CCC58233C5829BED9AEC99E582984088
:10CB08000CF582EE9BFEED9AFDEC99FC0FD5F0D664
:10CB1800E4CEFBE4CDFAE4CCF9A88222B800C1B98E
:10CB28000059BA002DEC8BF084CFCECDFCE5F0CBCC
:10CB3800F97818EF2FFFEE33FEED33FDEC33FCEB05
:10CB480033FB10D703994004EB99FB0FD8E5E4F9C0
:10CB5800FA227818EF2FFFEE33FEED33FDEC33FCAD
:10CB6800C933C910D7059BE99A4007EC9BFCE99AA1
:10CB7800F90FD8E0E4C9FAE4CCFB2275F010EF2FE6
:10CB8800FFEE33FEED33FDCC33CCC833C810D707E6
:10CB98009BEC9AE899400AED9BFDEC9AFCE899F821
:0ECBA8000FD5F0DAE4CDFBE4CCFAE4C8F922B4
:0DCBB600EF5BFFEE5AFEED59FDEC58FC223E
:0DCBC300EF4BFFEE4AFEED49FDEC48FC2271
:0DCBD000EF6BFFEE6AFEED69FDEC68FC22E4
:0DCBDD00CFF4CFCEF4CECDF4CDCCF4CC22ED
:10CBEA00EB9FF5F0EA9E42F0E99D42F0E89C45F0A1
:01CBFA002218
:10CBFB00E8600FECC313FCED13FDEE13FEEF13FF18
:03CC0B00D8F1223B
:10CC0E00E8600FEFC333FFEE33FEED33FDEC33FC84
:03CC1E00D8F12228
:0CCC2100E0FCA3E0FDA3E0FEA3E0FF2286
:0CCC2D00E0F8A3E0F9A3E0FAA3E0FB228A
:0CCC3900ECF0A3EDF0A3EEF0A3EFF0226E
:10CC4500A8828583F0D083D08212CC5C12CC5C1292
:10CC5500CC5C12CC5CE473E493A3C583C5F0C583B7
:10CC6500C8C582C8F0A3C583C5F0C583C8C582C839
:01CC7500229C
:09CC7600E0FBA3E0FAA3E0F922BF
:10CC7F00F8E0FBA3A3E0F925F0F0E582158270023E
:07CC8F001583E0FA38F022E2
:09CC9600EBF0A3EAF0A3E9F0229F
:10CC9F00BB010789828A8302CC765005E9F802CD61
:10CCAF0066BBFE05E9F802CD6F89828A8302CD78D3
:10CCBF00D083D082F8E4937012740193700DA3A304
:10CCCF0093F8740193F5828883E473740293686018
:06CCDF00EFA3A3A380DF18
:10CCE500EF4E6012EF60010EEDBB010B89828A8366
:10CCF500F0A3DFFCDEFA2289F05007F709DFFCA973
:0CCD0500F022BBFEFCF309DFFCA9F022C9
:10CD1100BC000BBE0029EF8DF084FFADF022E4CC06
:10CD2100F875F008EF2FFFEE33FEEC33FCEE9DECCF
:10CD3100984005FCEE9DFE0FD5F0E9E4CEFD22ED15
:10CD4100F8F5F0EE8420D21CFEADF075F008EF2F5F
:10CD5100FFED33FD4007985006D5F0F222C398FD50
:05CD61000FD5F0EA22ED
:09CD6600E6FB08E6FA08E6F922F2
:09CD6F00E2FB08E2FA08E2F922F5
:0CCD7800E493FB740193FA740293F92217
:00000001FF
